:020000040800F2
:1000000000300020B98F0008CD8D0008DB8D00087E
:10001000E18D0008E78D0008ED8D0008000000006C
:10002000000000000000000000000000F38D000848
:10003000018E0008000000000F8E00081D8E0008D1
:10004000099000080990000809900008099000082C
:10005000099000080990000809900008099000081C
:10006000099000080990000809900008099000080C
:1000700009900008099000080990000809900008FC
:1000800009900008099000080990000809900008EC
:1000900009900008099000080990000809900008DC
:1000A00009900008099000080990000809900008CC
:1000B000099000080990000800000000099000085D
:1000C00009900008000000000000000009900008EE
:1000D00000000000458E0008099000080990000803
:1000E00009900008099000080000000000000000CE
:1000F0000000000000000000000000000000000000
:1001000000000000000000000000000000000000EF
:10011000000000000000000009900008099000089D
:1001200000000000000000000000000000000000CF
:1001300000000000000000000000000000000000BF
:1001400009900008099000080000000009900008CC
:10015000099000080990000809900008099000081B
:10016000099000080990000800000000000000004D
:10017000000000000000000000000000000000007F
:080180000000000009900008D6
:1001900010B5054C237833B9044B13B10448AFF3C1
:1001A00000800123237010BD7400002000000000B7
:1001B00010AB000808B5034B1BB103490348AFF36C
:1001C000008008BD000000007800002010AB00088F
:1001D00001F0FF01102A2BDB10F0070F08D010F8F8
:1001E000013B013A8B422DD010F0070F42B3F6D1FC
:1001F000F0B441EA012141EA014122F007047FF015
:1002000000070023F0E80256083C85EA010586EA6B
:10021000010685FA47F5A3FA87F586FA47F6A5FAA7
:1002200087F68EB9EED1F0BC01F0FF0102F00702B3
:1002300032B110F8013B013A83EA010313B1F8D15E
:100240000020704701387047002D06BF354603383F
:10025000073815F0010F07D1013015F4807F02BF78
:10026000013015F4C03F0130F0BC0138704700BFC9
:1002700081F0004102E000BF83F0004330B54FEA57
:1002800041044FEA430594EA050F08BF90EA020FC4
:100290001FBF54EA000C55EA020C7FEA645C7FEA57
:1002A000655C00F0E2804FEA5454D4EB5555B8BF7A
:1002B0006D420CDD2C4480EA020281EA030382EAEB
:1002C000000083EA010180EA020281EA0303362D7D
:1002D00088BF30BD11F0004F4FEA01314FF4801C50
:1002E0004CEA113102D0404261EB410113F0004F62
:1002F0004FEA03334CEA133302D0524263EB430319
:1003000094EA050F00F0A780A4F10104D5F1200EB6
:100310000DDB02FA0EFC22FA05F2801841F1000111
:1003200003FA0EF2801843FA05F359410EE0A5F1E5
:1003300020050EF1200E012A03FA0EFC28BF4CF016
:10034000020C43FA05F3C01851EBE37101F00045CC
:1003500007D54FF0000EDCF1000C7EEB00006EEBD9
:100360000101B1F5801F1BD3B1F5001F0CD3490863
:100370005FEA30004FEA3C0C04F101044FEA4452BA
:1003800012F5800F80F09A80BCF1004F08BF5FEA41
:10039000500C50F1000041EB045141EA050130BD21
:1003A0005FEA4C0C404141EB010111F4801FA4F1C4
:1003B0000104E9D191F0000F04BF01460020B1FA19
:1003C00081F308BF2033A3F10B03B3F120020CDA51
:1003D0000C3208DD02F1140CC2F10C0201FA0CF02F
:1003E00021FA02F10CE002F11402D8BFC2F1200C94
:1003F00001FA02F120FA0CFCDCBF41EA0C0190404A
:10040000E41AA2BF01EB0451294330BD6FEA040492
:100410001F3C1CDA0C340EDC04F11404C4F120027D
:1004200020FA04F001FA02F340EA030021FA04F38F
:1004300045EA030130BDC4F10C04C4F1200220FAE6
:1004400002F001FA04F340EA0300294630BD21FA24
:1004500004F0294630BD94F0000F83F4801306BFEA
:1004600081F480110134013D4EE77FEA645C18BFDE
:100470007FEA655C29D094EA050F08BF90EA020F75
:1004800005D054EA000C04BF1946104630BD91EA6D
:10049000030F1EBF0021002030BD5FEA545C05D170
:1004A0004000494128BF41F0004130BD14F58004AF
:1004B0003CBF01F5801130BD01F0004545F0FE4123
:1004C00041F470014FF0000030BD7FEA645C1ABF58
:1004D000194610467FEA655C1CBF0B46024650EA8F
:1004E000013406BF52EA033591EA030F41F40021BB
:1004F00030BD00BF90F0000F04BF0021704730B541
:100500004FF4806404F132044FF000054FF0000115
:1005100050E700BF90F0000F04BF0021704730B5D6
:100520004FF4806404F1320410F0004548BF4042AB
:100530004FF000013EE700BF42004FEAE2014FEA00
:1005400031014FEA02701FBF12F07F4393F07F4FDB
:1005500081F06051704792F0000F14BF93F07F4F0D
:10056000704730B54FF4607401F0004521F0004150
:1005700020E700BF50EA010208BF704730B54FF0D6
:1005800000050AE050EA010208BF704730B511F0DB
:10059000004502D5404261EB41014FF4806404F113
:1005A00032045FEA915C3FF4DCAE4FF003025FEA95
:1005B000DC0C18BF03325FEADC0C18BF033202EB1D
:1005C000DC02C2F1200300FA03FC20FA02F001FA77
:1005D00003FE40EA0E0021FA02F11444C1E600BF16
:1005E00070B54FF0FF0C4CF4E06C1CEA11541DBFC9
:1005F0001CEA135594EA0C0F95EA0C0F00F0DEF894
:100600002C4481EA030621EA4C5123EA4C5350EA78
:10061000013518BF52EA033541F4801143F48013C9
:1006200038D0A0FB02CE4FF00005E1FB02E506F05A
:100630000042E0FB03E54FF00006E1FB03569CF0AF
:10064000000F18BF4EF0010EA4F1FF04B6F5007FB5
:1006500064F5407404D25FEA4E0E6D4146EB060627
:1006600042EAC62141EA55514FEAC52040EA5E50B0
:100670004FEACE2EB4F1FD0C88BFBCF5E06F1ED85A
:10068000BEF1004F08BF5FEA500E50F1000041EB91
:10069000045170BD06F0004646EA010140EA02003E
:1006A00081EA0301B4EB5C04C2BFD4EB0C0541EA60
:1006B000045170BD41F480114FF0000E013C00F375
:1006C000AB8014F1360FDEBF002001F0004170BD99
:1006D000C4F10004203C35DA0C341BDC04F11404B2
:1006E000C4F1200500FA05F320FA04F001FA05F23E
:1006F00040EA020001F0004221F0004110EBD3700B
:1007000021FA04F642EB06015EEA430E08BF20EA36
:10071000D37070BDC4F10C04C4F1200500FA04F3D9
:1007200020FA05F001FA04F240EA020001F000416B
:1007300010EBD37041F100015EEA430E08BF20EADE
:10074000D37070BDC4F1200500FA05F24EEA020E26
:1007500020FA04F301FA05F243EA020321FA04F055
:1007600001F0004121FA04F220EA020000EBD3700C
:100770005EEA430E08BF20EAD37070BD94F0000F0C
:100780000FD101F00046400041EB010111F4801F40
:1007900008BF013CF7D041EA060195F0000F18BFF1
:1007A000704703F00046520043EB030313F4801F2D
:1007B00008BF013DF7D043EA0603704794EA0C0FE7
:1007C0000CEA135518BF95EA0C0F0CD050EA4106FD
:1007D00018BF52EA4306D1D181EA030101F000417A
:1007E0004FF0000070BD50EA410606BF10461946A2
:1007F00052EA430619D094EA0C0F02D150EA0136AE
:1008000013D195EA0C0F05D152EA03361CBF1046EE
:1008100019460AD181EA030101F0004141F0FE418D
:1008200041F470014FF0000070BD41F0FE4141F411
:10083000780170BD70B54FF0FF0C4CF4E06C1CEA11
:1008400011541DBF1CEA135594EA0C0F95EA0C0FC6
:1008500000F0A7F8A4EB050481EA030E52EA033581
:100860004FEA013100F088804FEA03334FF08055A2
:1008700045EA131343EA12634FEA022245EA1115CF
:1008800045EA10654FEA00260EF000419D4208BF80
:10089000964244F1FD0404F5407402D25B084FEA2D
:1008A0003202B61A65EB03055B084FEA32024FF4D9
:1008B00080104FF4002CB6EB020E75EB030E22BF36
:1008C000B61A754640EA0C005B084FEA3202B6EBF6
:1008D000020E75EB030E22BFB61A754640EA5C00A5
:1008E0005B084FEA3202B6EB020E75EB030E22BF35
:1008F000B61A754640EA9C005B084FEA3202B6EB36
:10090000020E75EB030E22BFB61A754640EADC00F4
:1009100055EA060E18D04FEA051545EA16754FEA56
:1009200006164FEAC30343EA52734FEAC2025FEA74
:100930001C1CC0D111F4801F0BD141EA00014FF003
:1009400000004FF0004CB6E711F4801F04BF0143D4
:100950000020B4F1FD0C88BFBCF5E06F3FF6AFAEF0
:10096000B5EB030C04BFB6EB020C5FEA500C50F180
:10097000000041EB045170BD0EF0004E4EEA113103
:1009800014EB5C04C2BFD4EB0C0541EA045170BD0A
:1009900041F480114FF0000E013C90E645EA060E4E
:1009A0008DE60CEA135594EA0C0F08BF95EA0C0F7C
:1009B0003FF43BAF94EA0C0F0AD150EA01347FF4C4
:1009C00034AF95EA0C0F7FF425AF104619462CE79B
:1009D00095EA0C0F06D152EA03353FF4FDAE1046FE
:1009E000194622E750EA410618BF52EA43067FF44F
:1009F000C5AE50EA41047FF40DAF52EA43057FF4DF
:100A0000EBAE12E74FF0FF3C06E000BF4FF0010CE9
:100A100002E000BF4FF0010C4DF804CD4FEA410C4D
:100A20007FEA6C5C4FEA430C18BF7FEA6C5C1BD01A
:100A300001B050EA410C0CBF52EA430C91EA030F9B
:100A400002BF90EA020F0020704710F1000F91EAF8
:100A5000030F58BF994208BF90422CBFD8176FEAC6
:100A6000E37040F0010070474FEA410C7FEA6C5C94
:100A700002D150EA013C07D14FEA430C7FEA6C5C9B
:100A8000D6D152EA033CD3D05DF8040B704700BFC7
:100A90008446104662468C461946634600E000BF15
:100AA00001B5FFF7B7FF002848BF10F1000F01BDE7
:100AB0004DF808EDFFF7F4FF0CBF012000205DF8B2
:100AC00008FB00BF4DF808EDFFF7EAFF34BF012037
:100AD00000205DF808FB00BF4DF808EDFFF7E0FFD0
:100AE00094BF012000205DF808FB00BF4DF808ED21
:100AF000FFF7CEFF94BF012000205DF808FB00BF88
:100B00004DF808EDFFF7C4FF34BF012000205DF869
:100B100008FB00BF4FEA410C7FEA6C5C02D150EA4F
:100B2000013C0AD14FEA430C7FEA6C5C02D152EAE5
:100B3000033C02D14FF0000070474FF001007047B6
:100B40004FEA410212F5001215D211D56FF47873F5
:100B5000B3EB625212D94FEAC12343F0004343EA98
:100B6000505311F0004F23FA02F018BF4042704773
:100B70004FF00000704750EA013005D111F00040FD
:100B800008BF6FF0004070474FF00000704700BF93
:100B90004FEA4102B2F1E04324BFB3F5001CDCF19F
:100BA000FE5C0DD901F0004C4FEAC0024CEA5070D7
:100BB000B2F1004F40EB830008BF20F00100704706
:100BC00011F0804F21D113F13872BCBF01F0004009
:100BD000704741F480114FEA5252C2F11802C2F13B
:100BE000200C10FA0CF320FA02F018BF40F00100BC
:100BF0004FEAC1234FEAD32303FA0CFC40EA0C006E
:100C000023FA02F34FEA4303CCE77FEA625307D1AA
:100C100050EA01331EBF4FF0FE4040F440007047E1
:100C200001F0004040F0FE4040F40000704700BF7B
:100C30007BB972B90029BEBF00204FF0004106E029
:100C400008BF00281CBF6FF000414FF0FF3000F0DC
:100C5000ADB9ADF1080C6DE904CE002909DB002B1C
:100C60001ADB00F035F8DDF804E0DDE9022304B01A
:100C70007047404261EB4101002B1BDB00F028F87C
:100C8000DDF804E0DDE9022304B0404261EB4101FC
:100C9000524263EB43037047524263EB430300F05D
:100CA00017F8DDF804E0DDE9022304B0404261EB0F
:100CB00041017047524263EB430300F009F8DDF84D
:100CC00004E0DDE9022304B0524263EB43037047C2
:100CD0002DE9F0478C460D460446089E002B51D165
:100CE0008A4217466DD9B2FA82FEBEF1000F0BD0D0
:100CF000CEF1200C01FA0EF520FA0CFC02FA0EF7E8
:100D00004CEA050C00FA0EF44FEA174A250CBCFB1E
:100D1000FAF81FFA87F90AFB18CC45EA0C4508FBDC
:100D200009F3AB420AD9ED1908F1FF3280F02381B3
:100D3000AB4240F22081A8F102083D44ED1AA4B272
:100D4000B5FBFAF00AFB105544EA054400FB09F92B
:100D5000A14509D9E41900F1FF3380F00A81A145CA
:100D600040F2078102383C44A4EB090440EA084001
:100D70000021002E61D024FA0EF400233460736049
:100D8000BDE8F0878B4207D9002E54D0002186E8B9
:100D900021000846BDE8F087B3FA83F1002940F04E
:100DA0008E80AB4202D3824200F2FA80841A65EB55
:100DB00003050120AC46002E3FD086E81010BDE8A8
:100DC000F08712B90127B7FBF2F7B7FA87FEBEF139
:100DD000000F34D1EB1B3A0C1FFA87FC0121B3FB47
:100DE000F2F8250C02FB183345EA03450CFB08F327
:100DF000AB4207D9ED1908F1FF3002D2AB4200F245
:100E0000D1808046ED1AA3B2B5FBF2F002FB10557B
:100E100043EA05440CFB00FCA44507D9E41900F1A2
:100E2000FF3302D2A44500F2B8801846A4EB0C04AC
:100E300040EA08409DE731463046BDE8F087CEF1F4
:100E4000200405FA0EF307FA0EF720FA04F83A0C1C
:100E500025FA04F448EA0308B4FBF2F14FEA184516
:100E600002FB11441FFA87FC45EA044501FB0CF321
:100E7000AB4200FA0EF409D9ED1901F1FF3080F010
:100E80008A80AB4240F2878002393D44EB1A1FFA58
:100E900088F5B3FBF2F002FB103345EA034500FB93
:100EA0000CF3AB4207D9ED1900F1FF386FD2AB421A
:100EB0006DD902383D44EB1A40EA01418FE7C1F198
:100EC000200722FA07F88B4005FA01F448EA0303E9
:100ED00020FA07FE4FEA134CFD404EEA040EB5FB24
:100EE000FCF94FEA1E440CFB19551FFA83F844EA3B
:100EF000054509FB08F4AC4202FA01F200FA01FAD6
:100F000008D9ED1809F1FF3043D2AC4241D9A9F11B
:100F100002091D442D1B1FFA8EFEB5FBFCF00CFBD5
:100F200010554EEA054400FB08F8A04507D9E4181F
:100F300000F1FF3529D2A04527D902381C4440EAE8
:100F40000940A4EB0804A0FB02894C45C6464D4667
:100F500015D312D056B1BAEB0E0364EB050404FAB4
:100F600007F7CB401F43CC40376074600021BDE8D9
:100F7000F0871846F8E69046E0E6C245EAD2B8EBBC
:100F8000020E69EB03050138E4E72846D7E740463F
:100F900091E78146BEE7014678E702383C4445E7E1
:100FA000084608E7A8F102083D442BE7704700BF58
:100FB00080B500AF084A084B1B6843F0100313606C
:100FC000032000F0DBFF002000F008F807F0F0FD40
:100FD0000023184680BD00BF0020024080B582B0CB
:100FE00000AF7860124B1A68124B1B7819464FF409
:100FF0007A73B3FBF1F3B2FBF3F3184600F0F3FF9F
:101000000346002B01D001230EE07B680F2B0AD88A
:10101000002279684FF0FF3000F0BBFF064A7B6882
:101020001360002300E0012318460837BD4680BD49
:1010300008000020040000200000002080B400AF61
:10104000064B1B781A46064B1B681344044A136070
:1010500000BFBD465DF8047B704700BF0400002060
:10106000D000002080B400AF034B1B681846BD467B
:101070005DF8047B704700BFD000002080B584B0CD
:1010800000AF7860FFF7EEFFB8607B68FB60FB683D
:10109000B3F1FF3F05D0094B1B781A46FB68134498
:1010A000FB6000BFFFF7DEFF0246BB68D21AFB6899
:1010B0009A42F7D300BF1037BD4680BD0400002020
:1010C00080B59CB000AF7860002387F86F300023B4
:1010D000BB660023FB607B68002B01D1012370E11C
:1010E0007B681B69002B7B685B6C03F01003002B93
:1010F00076D17B685B6C002B52D17B6800229A64AE
:101100007B6800221A657B680022DA647B68002213
:1011100083F84020786807F06FFD7B681B689B6848
:1011200003F08053002B3BD1786800F0FDFD0346AF
:1011300087F86F307B685B6C03F01003002B2FD1B6
:1011400097F86F30002B2BD17B685B6C23F48853AE
:1011500023F0020343F002027B685A647B681B6839
:101160007A681268926822F040529A607B681B6825
:101170007A681268926842F080529A60934B1B68BA
:10118000934AA2FB03239A0C13469B0013445B0073
:10119000FB6002E0FB68013BFB60FB68002BF9D1C0
:1011A0007B681B689B6803F08053002B07D07B682B
:1011B0001B689B6803F00053B3F1005F10D17B689C
:1011C0005B6C23F0120343F010027B685A647B6867
:1011D0009B6C43F001027B689A64012387F86F30AF
:1011E0007B685B6C03F01003002B40F0DD8097F808
:1011F0006F30002B40F0D8807B681B689B6803F041
:101200000403002B40F0D0807B685B6C23F4817377
:1012100043F002027B685A646E4B7B667B681B68F6
:10122000B3F1A04F02D16C4B3B6102E04FF0A04301
:101230003B617B681B689B6803F00303012B08D1AB
:101240007B681B681B6803F00103012B01D101239C
:1012500000E00023002B1CD13B69002B10D03B6920
:101260009B6803F00303012B07D13B691B6803F064
:101270000103012B01D1012300E00023002B08D141
:101280007B6E9B6823F440327B685B681A437B6EFD
:101290009A607B68DB695A037B689B6B012B02D0E9
:1012A0004FF4805300E000231A437B68DB681A4345
:1012B0007B689B681343BA6E1343BB667B685B6AAB
:1012C000012B1BD17B68DB69002B09D17B689B6AF2
:1012D000013B5A04BB6E134343F48033BB660DE0FD
:1012E0007B685B6C23F0220343F020027B685A6426
:1012F0007B689B6C43F001027B689A647B68DB6AC5
:10130000012B07D07B68DA6A7B681B6B1343BA6ECC
:101310001343BB667B681B689B6803F00C03002BC0
:1013200013D17B681A687B681B68DB6823F48043F1
:1013300023F00203D3607B689B699A037B685B6B35
:101340005B001343BA6E1343BB667B681A687B6805
:101350001B68D968214B0B40B96E0B43D3607B6887
:101360001B69012B0CD17B681B687A681268126BB1
:1013700022F00F017A68126A013A0A431A6307E001
:101380007B681B687A681268126B22F00F021A637E
:101390007B6800229A647B685B6C23F0030343F054
:1013A00001027B685A640AE07B685B6C23F01203DD
:1013B00043F010027B685A64012387F86F3097F876
:1013C0006F3018467037BD4680BD00BF0800002052
:1013D00083DE1B43000300500001005007C0F0FFF4
:1013E00080B584B000AF78600023FB737B681B6816
:1013F0009B6803F00403002B40F09C807B6893F80B
:101400004030012B01D1022397E07B68012283F851
:101410004020786800F02AFC0346FB73FB7B002B1E
:1014200040F083807B685B6C23F4706323F00103DE
:1014300043F480727B685A64424B9B6803F01F033D
:10144000002B04D07B681B68B3F1A04F15D17B68DB
:101450005B6C23F480127B685A647B681B68DB68D2
:1014600003F00073002B27D07B685B6C23F44053A0
:1014700043F480527B685A641EE07B685B6C43F4E3
:1014800080127B685A647B681B68B3F1A04F04D05C
:101490007B681B682C4A93420ED14FF0A043DB6857
:1014A00003F00073002B07D07B685B6C23F4405380
:1014B00043F480527B685A647B685B6C03F480530E
:1014C000B3F5805F06D17B689B6C23F006027B68D6
:1014D0009A6402E07B6800229A647B68002283F8A9
:1014E00040207B681B681C221A60164B9B6803F027
:1014F0001F03002B10D0134B9B6803F01F03052B19
:101500000AD0104B9B6803F01F03092B04D07B68A3
:101510001B68B3F1A04F0FD17B681B687A68126813
:10152000926842F004029A6006E07B68002283F829
:10153000402001E00223FB73FB7B18461037BD46B9
:1015400080BD00BF000300500001005080B483B094
:1015500000AF78607B681B681B6C18460C37BD4673
:101560005DF8047B7047000090B49CB000AF7860D9
:101570003960002387F86F300023FB607B6893F8A5
:101580004030012B01D10223A3E27B68012283F8C2
:1015900040207B681B689B6803F00403002B40F02D
:1015A00087823B685B68042B1CD87B6819687B6862
:1015B0001B68186B3B685A6813465B0013445B005A
:1015C0001A461F239340DB4318403B681C683B6866
:1015D0005A6813465B0013445B0004FA03F30343A9
:1015E0000B6363E03B685B68092B1ED87B68196856
:1015F0007B681B68586B3B685A6813465B00134452
:101600005B001E3B1F2202FA03F3DB4318403B68DA
:101610001C683B685A6813465B0013445B001E3B22
:1016200004FA03F303434B6340E03B685B680E2B13
:101630001ED87B6819687B681B68986B3B685A6882
:1016400013465B0013445B003C3B1F2202FA03F38A
:10165000DB4318403B681C683B685A6813465B00D4
:1016600013445B003C3B04FA03F303438B631DE02C
:101670007B6819687B681B68D86B3B685A6813469F
:101680005B0013445B005A3B1F2202FA03F3DB4367
:1016900018403B681C683B685A6813465B0013445B
:1016A0005B005A3B04FA03F30343CB637B681B687C
:1016B0009B6803F00C03002B40F0E5803B681B683F
:1016C000092B1CD97B6819687B681B6898693B6883
:1016D0001A6813465B0013441E3B072202FA03F309
:1016E000DB4318403B689C683B681A6813465B0004
:1016F00013441E3B04FA03F303438B6119E07B6838
:1017000019687B681B6858693B681A6813465B0058
:101710001344072202FA03F3DB4318403B689C683A
:101720003B681A6813465B00134404FA03F303434F
:101730004B613B685A697B681B68DB68DB0803F018
:1017400003035B0002FA03F3BB663B681B69013BC2
:10175000032B4FD801A252F823F000BF6D170008E9
:101760008F170008B1170008D31700087B681A68A4
:101770007B681B68196E9C4B0B40396809688806AA
:10178000B96E01430B4343F0004313667BE07B6873
:101790001A687B681B68596E934B0B40396809685F
:1017A0008806B96E01430B4343F0004353666AE079
:1017B0007B681A687B681B68996E8B4B0B40396895
:1017C00009688806B96E01430B4343F000439366F2
:1017D00059E07B681A687B681B68D96E824B0B40A6
:1017E000396809688806B96E01430B4343F000432A
:1017F000D36648E07B681B681B6E03F0F8423B68C9
:101800001B689B069A4207D17B681B687A6812683E
:10181000126E22F000421A667B681B685B6E03F052
:10182000F8423B681B689B069A4207D17B681B689D
:101830007A681268526E22F000425A667B681B6812
:101840009B6E03F0F8423B681B689B069A4207D1E7
:101850007B681B687A681268926E22F000429A6672
:101860007B681B68DB6E03F0F8423B681B689B06D5
:101870009A4207D17B681B687A681268D26E22F0A0
:101880000042DA6600BF7B681B689B6803F00303B5
:10189000012B08D17B681B681B6803F00103012B37
:1018A00001D1012300E00023002B40F00C813B68B4
:1018B000DB68012B0FD07B681B687A681268D2F84E
:1018C000B0103A681268012000FA02F2D2430A40CE
:1018D000C3F8B0204AE07B681B687A681268D2F8C7
:1018E000B0103A681268012000FA02F20A43C3F805
:1018F000B0203B681B68092B1CD97B6819687B6882
:101900001B6898693B681A6813465B0013441B3BCD
:10191000072202FA03F3DB4318403B689C683B68EC
:101920001A6813465B0013441B3B04FA03F303439A
:101930008B611BE07B6819687B681B6858693B6892
:101940001B685A1C13465B001344072202FA03F378
:10195000DB4318403B689C683B681B685A1C134675
:101960005B00134404FA03F303434B611F4B7B6694
:101970003B681B68102B05D17B6E9B6803F400034A
:10198000002B15D03B681B68112B05D17B6E9B6823
:1019900003F08073002B0BD03B681B68122B40F0C8
:1019A00092807B6E9B6803F48003002B40F08B8059
:1019B0007B681B68B3F1A04F02D10D4B3B6102E085
:1019C0004FF0A0433B617B681B689B6803F00303F7
:1019D000012B0FD17B681B681B6803F00103012BEF
:1019E00008D1012307E000BF00F0FF83000300508F
:1019F000000100500023002B50D13B69002B10D078
:101A00003B699B6803F00303012B07D13B691B680B
:101A100003F00103012B01D1012300E00023002B7F
:101A20003CD13B681B68102B1DD17B681B68B3F150
:101A3000A04F18D17B6E9B6843F400027B6E9A60C6
:101A4000264B1B68264AA2FB03239A0C13469B00D5
:101A500013445B00FB6002E0FB68013BFB60FB683A
:101A6000002BF9D12EE03B681B68112B0BD17B6852
:101A70001B68B3F1A04F06D17B6E9B6843F0807268
:101A80007B6E9A601EE03B681B68122B1AD17B6E3E
:101A90009B6843F480027B6E9A6013E07B685B6C0A
:101AA00043F020027B685A64012387F86F300AE014
:101AB0007B685B6C43F020027B685A64012387F8E3
:101AC0006F3000E000BF7B68002283F8402097F869
:101AD0006F3018467037BD4690BC70470800002034
:101AE00083DE1B4380B49BB000AF78603960002375
:101AF00087F867307B681B68B3F1A04F02D1594B60
:101B0000FB6002E04FF0A043FB60FB68002B01D1BB
:101B10000123A1E07B6893F84030012B01D102231F
:101B20009AE07B68012283F840207B681B689B68F1
:101B300003F00403002B7ED1FB689B6803F00403D1
:101B4000002B78D1484B3B663B681B68002B3FD08D
:101B50003B6E9B6823F460423B6859687B685B6B13
:101B60005B030B431A433B6E9A607B681B689B6860
:101B700003F00303012B08D17B681B681B6803F08B
:101B80000103012B01D1012300E00023002B5CD1D4
:101B9000FB689B6803F00303012B07D1FB681B68FC
:101BA00003F00103012B01D1012300E00023002BEE
:101BB0004BD13B6E9B6823F4716323F00F033A68AB
:101BC00011683A6892680A431A433B6E9A603CE097
:101BD0003B6E9B6823F460423B6E9A607B681B6897
:101BE0009B6803F00303012B08D17B681B681B680B
:101BF00003F00103012B01D1012300E00023002B9E
:101C000023D1FB689B6803F00303012B07D1FB681A
:101C10001B6803F00103012B01D1012300E0002325
:101C2000002B12D13B6E9B6823F4716323F00F03EA
:101C30003A6E936009E07B685B6C43F020027B683E
:101C40005A64012387F8673000E000BF7B680022F8
:101C500083F8402097F8673018466C37BD465DF82A
:101C6000047B7047000100500003005080B584B031
:101C700000AF78600023FB607B681B689B6803F003
:101C80000303012B08D17B681B681B6803F0010369
:101C9000012B01D1012300E00023002B3CD17B6804
:101CA0001B689A681F4B1340002B0DD07B685B6C40
:101CB00043F010027B685A647B689B6C43F001021E
:101CC0007B689A64012328E07B681B687A68126845
:101CD000926842F001029A60FFF7C4F9F86014E0DC
:101CE000FFF7C0F90246FB68D31A022B0DD97B68B7
:101CF0005B6C43F010027B685A647B689B6C43F01A
:101D000001027B689A64012307E07B681B681B68FB
:101D100003F00103012BE3D1002318461037BD4621
:101D200080BD00BF3F00008080B584B000AF786008
:101D30000023FB607B681B689B6803F00303012B97
:101D400008D17B681B681B6803F00103012B01D1DC
:101D5000012300E00023002B40D07B681B689B68B8
:101D600003F00D03012B0FD17B681B687A681268A2
:101D7000926842F002029A607B681B6803221A6034
:101D8000FFF770F9F86022E07B685B6C43F01002AB
:101D90007B685A647B689B6C43F001027B689A64A1
:101DA00001231CE0FFF75EF90246FB68D31A022B01
:101DB0000DD97B685B6C43F010027B685A647B68CA
:101DC0009B6C43F001027B689A64012307E07B6807
:101DD0001B689B6803F00103012BE3D00023184626
:101DE0001037BD4680BD000080B485B000AF78607C
:101DF0007B6803F00703FB600C4BDB68BB60BA68D1
:101E00004FF6FF031340BB60FB681A02BB68134325
:101E100043F0BF6343F40033BB60044ABB68D36044
:101E200000BF1437BD465DF8047B704700ED00E04D
:101E300080B400AF044BDB681B0A03F007031846AD
:101E4000BD465DF8047B704700ED00E080B483B0D0
:101E500000AF0346FB71094997F907305B09FA792E
:101E600002F01F02012000FA02F241F8232000BF15
:101E70000C37BD465DF8047B704700BF00E100E011
:101E800080B483B000AF03463960FB7197F9073027
:101E9000002B0BDA0D49FB7903F00F03043B3A6882
:101EA000D2B21201D2B20B441A7609E0084997F96E
:101EB00007303A68D2B21201D2B20B4483F8002341
:101EC00000BF0C37BD465DF8047B704700ED00E0B5
:101ED00000E100E080B489B000AFF860B9607A60DA
:101EE000FB6803F00703FB61FB69C3F10703042BE5
:101EF00028BF0423BB61FB690433062B02D9FB69AD
:101F0000033B00E000237B610122BB6902FA03F37B
:101F10005A1EBB681A407B699A4001217B6901FA0D
:101F200003F3591E7B680B40134318462437BD4604
:101F30005DF8047B7047000080B582B000AF786028
:101F40007B68013BB3F1807F01D301230FE00A4A94
:101F50007B68013B53600F214FF0FF30FFF790FF8C
:101F6000054B00229A60044B07221A600023184692
:101F70000837BD4680BD00BF10E000E080B582B0EC
:101F800000AF78607868FFF72FFF00BF0837BD46C5
:101F900080BD80B586B000AF0346B9607A60FB7340
:101FA00000237B61FFF744FF78617A68B96878693C
:101FB000FFF790FF024697F90F3011461846FFF7DA
:101FC0005FFF00BF1837BD4680BD80B582B000AF4F
:101FD0000346FB7197F907301846FFF737FF00BF3C
:101FE0000837BD4680BD80B582B000AF78607868A4
:101FF000FFF7A2FF034618460837BD4680BD80B5EF
:1020000084B000AF78600023FB737B6893F82130C5
:10201000022B05D07B6804229A630123FB7327E01F
:102020007B681B687A681268126822F00E021A60D8
:102030007B681B687A681268126822F001021A60D5
:102040007B68DB6B7A68126C012101FA02F25A603C
:102050007B68012283F821207B68002283F82020FE
:102060007B685B6B002B03D07B685B6B7868984761
:10207000FB7B18461037BD4680BD000080B487B09A
:1020800000AF7860396000237B610023FB60002390
:102090003B614EE13B681A6801217B6901FA03F359
:1020A0001340FB60FB68002B00F040813B685B68DD
:1020B000022B03D03B685B68122B23D17B69DA08C3
:1020C0007B68083253F822303B617B6903F00703D9
:1020D0009B000F2202FA03F3DB433A6913403B6192
:1020E0003B681A697B6903F007039B0002FA03F35C
:1020F0003A6913433B617B69DA087B6808323969C6
:1021000043F822107B681B683B617B695B000322FC
:1021100002FA03F3DB433A6913403B613B685B68B7
:1021200003F003027B695B0002FA03F33A6913438D
:102130003B617B683A691A603B685B68012B0BD096
:102140003B685B68022B07D03B685B68112B03D0B0
:102150003B685B68122B30D17B689B683B617B6975
:102160005B00032202FA03F3DB433A6913403B614D
:102170003B68DA687B695B0002FA03F33A69134350
:102180003B617B683A699A607B685B683B610122CE
:102190007B6902FA03F3DB433A6913403B613B6816
:1021A0005B681B0903F001027B6902FA03F33A69D9
:1021B00013433B617B683A695A607B68DB683B612B
:1021C0007B695B00032202FA03F3DB433A691340A5
:1021D0003B613B689A687B695B0002FA03F33A69EA
:1021E00013433B617B683A69DA603B685B6803F0E4
:1021F0008053002B00F09A80554A554B9B6943F061
:1022000001039361524B9B6903F00103BB60BB6800
:10221000504A7B699B08023352F823303B617B694B
:1022200003F003039B000F2202FA03F3DB433A6936
:1022300013403B617B68B3F1904F13D07B68464AF3
:1022400093420DD07B68454A934207D07B68444A4D
:10225000934201D1032306E0052304E0022302E0B8
:10226000012300E000237A6902F003029200934008
:102270003A6913433B6137497B699B0802333A69EA
:1022800041F82320374B1B683B61FB68DB433A690D
:1022900013403B613B685B6803F48033002B03D041
:1022A0003A69FB6813433B612E4A3B6913602D4B2F
:1022B0005B683B61FB68DB433A6913403B613B6809
:1022C0005B6803F40033002B03D03A69FB681343C7
:1022D0003B61244A3B695360224B9B683B61FB682E
:1022E000DB433A6913403B613B685B6803F480134E
:1022F000002B03D03A69FB6813433B61194A3B69E1
:102300009360184BDB683B61FB68DB433A69134021
:102310003B613B685B6803F40013002B03D03A6910
:10232000FB6813433B610F4A3B69D3607B69013310
:102330007B613B681A687B6922FA03F3002B7FF408
:10234000A9AE00BF1C37BD465DF8047B704700BFD7
:10235000001002400000014000040048000800484E
:10236000000C00480004014080B483B000AF7860E6
:102370000B467B8013467B707B78002B03D07A88DA
:102380007B689A6102E07A887B689A6200BF0C37AA
:10239000BD465DF8047B704780B582B000AF7860C1
:1023A0007B68002B01D1012380E07B6893F84130EA
:1023B000DBB2002B06D17B68002283F840207868CE
:1023C00006F056FC7B68242283F841207B681B685A
:1023D0007A681268126822F001021A607B681B6832
:1023E0007A68526822F070621A617B681B687A68AA
:1023F0001268926822F400429A607B68DB68012BC5
:1024000007D17B681B687A68926842F400429A6040
:1024100006E07B681B687A68926842F404429A601E
:102420007B68DB68022B04D17B681B684FF4006279
:102430005A607B681A687B681B685B6843F00073AE
:1024400043F4004353607B681B687A681268D26863
:1024500022F40042DA607B681B687A6811697A6846
:10246000526911437A68926912020A43DA607B6802
:102470001B687A68D1697A68126A0A431A607B68B5
:102480001B687A681268126842F001021A607B6861
:1024900000225A647B68202283F841207B68002256
:1024A0001A637B68002283F842200023184608370D
:1024B000BD4680BD80B588B002AFF86008461146C1
:1024C0001A4603467B810B463B811346FB80002363
:1024D0007B61FB6893F84130DBB2202B40F009812F
:1024E0003B6A002B02D0BB8C002B01D1012301E100
:1024F000FB6893F84030012B01D10223FAE0FB681E
:10250000012283F84020FEF7ADFD78617B690093DE
:10251000192301224FF40041F86800F0FBFA03464A
:10252000002B01D00323E5E0FB68212283F8412042
:10253000FB68402283F84220FB6800225A64FB6853
:102540003A6A5A62FB68BA8C5A85FB6800225A6361
:10255000F8883A8979897B690193BB6A00930346BD
:10256000F86800F0F3F90346002B0FD0FB685B6CB2
:10257000042B05D1FB68002283F840200123B9E039
:10258000FB68002283F840200323B3E0FB685B8DE7
:102590009BB2FF2B0ED9FB68FF221A85FB681B8DAF
:1025A000DAB27989002300934FF08073F86800F065
:1025B000C5FB0FE0FB685B8D9AB2FB681A85FB6870
:1025C0001B8DDAB27989002300934FF00073F8680D
:1025D00000F0B4FB7A69B96AF86800F0D5FA0346EE
:1025E000002B07D0FB685B6C042B01D1012381E039
:1025F00003237FE0FB681A68FB685B6A581CF96874
:1026000048621B789362FB685B8D9BB2013B9AB278
:10261000FB685A85FB681B8D013B9AB2FB681A85E3
:10262000FB681B8D002B35D1FB685B8D9BB2002BAB
:1026300030D07B690093BB6A00228021F86800F0EB
:1026400069FA0346002B01D0032353E0FB685B8D3E
:102650009BB2FF2B0ED9FB68FF221A85FB681B8DEE
:10266000DAB27989002300934FF08073F86800F0A4
:1026700065FB0FE0FB685B8D9AB2FB681A85FB680F
:102680001B8DDAB27989002300934FF00073F8684C
:1026900000F054FBFB685B8D9BB2002B9AD17A69EA
:1026A000B96AF86800F0B0FA0346002B07D0FB685F
:1026B0005B6C042B01D101231CE003231AE0FB68AF
:1026C0001B682022DA61FB681A68FB681B6859687E
:1026D0000A4B0B405360FB68202283F84120FB68C3
:1026E000002283F84220FB68002283F84020002368
:1026F00000E0022318461837BD4680BD00E800FE02
:1027000080B588B002AFF860084611461A46034605
:102710007B810B463B811346FB8000237B61FB687A
:1027200093F84130DBB2202B40F007813B6A002B4D
:1027300002D0BB8C002B01D10123FFE0FB6893F892
:102740004030012B01D10223F8E0FB68012283F81D
:102750004020FEF787FC78617B69009319230122F2
:102760004FF40041F86800F0D5F90346002B01D082
:102770000323E3E0FB68222283F84120FB68402228
:1027800083F84220FB6800225A64FB683A6A5A6266
:10279000FB68BA8C5A85FB6800225A63F8883A892C
:1027A00079897B690193BB6A00930346F86800F05E
:1027B0002DF90346002B0FD0FB685B6C042B05D171
:1027C000FB68002283F840200123B7E0FB68002269
:1027D00083F840200323B1E0FB685B8D9BB2FF2BA5
:1027E0000ED9FB68FF221A85FB681B8DDAB2798946
:1027F000544B00934FF08073F86800F09FFA0FE09D
:10280000FB685B8D9AB2FB681A85FB681B8DDAB298
:1028100079894C4B00934FF00073F86800F08EFA02
:102820007B690093BB6A00220421F86800F072F90A
:102830000346002B01D0032380E0FB685B6A591C30
:10284000FA685162FA681268526AD2B21A70FB686A
:102850001B8D013B9AB2FB681A85FB685B8D9BB2AE
:10286000013B9AB2FB685A85FB681B8D002B35D162
:10287000FB685B8D9BB2002B30D07B690093BB6AF9
:1028800000228021F86800F045F90346002B01D0B2
:10289000032353E0FB685B8D9BB2FF2B0ED9FB68D3
:1028A000FF221A85FB681B8DDAB279890023009319
:1028B0004FF08073F86800F041FA0FE0FB685B8D21
:1028C0009AB2FB681A85FB681B8DDAB279890023FE
:1028D00000934FF00073F86800F030FAFB685B8DEE
:1028E0009BB2002B9CD17A69B96AF86800F08CF928
:1028F0000346002B07D0FB685B6C042B01D101233E
:102900001CE003231AE0FB681B682022DA61FB68E5
:102910001A68FB681B6859680B4B0B405360FB68D7
:10292000202283F84120FB68002283F84220FB68C4
:10293000002283F84020002300E0022318461837C5
:10294000BD4680BD0024008000E800FE80B586B052
:1029500002AFF860084611461A4603467B810B46D3
:102960003B811346FB80FB88DAB27989264B0093C2
:102970004FF08073F86800F0E1F9FA69B969F86816
:1029800000F002F90346002B07D0FB685B6C042BB8
:1029900001D1012334E0032332E0FB88012B05D170
:1029A000FB681B683A89D2B29A621BE0FB681B681D
:1029B0003A89120A92B2D2B29A62FA69B969F8688F
:1029C00000F0E2F80346002B07D0FB685B6C042B99
:1029D00001D1012314E0032312E0FB681B683A894C
:1029E000D2B29A62FB690093BB6900228021F86829
:1029F00000F090F80346002B01D0032300E00023F1
:102A000018461037BD4680BD0020008080B586B0D6
:102A100002AFF860084611461A4603467B810B4612
:102A20003B811346FB80FB88DAB27989264B009301
:102A30000023F86800F082F9FA69B969F86800F0D3
:102A4000A3F80346002B07D0FB685B6C042B01D175
:102A5000012334E0032332E0FB88012B05D1FB681E
:102A60001B683A89D2B29A621BE0FB681B683A89FC
:102A7000120A92B2D2B29A62FA69B969F86800F0A1
:102A800083F80346002B07D0FB685B6C042B01D155
:102A9000012314E0032312E0FB681B683A89D2B2D9
:102AA0009A62FB690093BB6900224021F86800F03C
:102AB00031F80346002B01D0032300E00023184621
:102AC0001037BD4680BD00BF0020008080B483B0B9
:102AD00000AF78607B681B689B6903F00203022BE0
:102AE00003D17B681B6800229A627B681B689B6924
:102AF00003F00103012B07D07B681B687A6812681A
:102B0000926942F001029A6100BF0C37BD465DF840
:102B1000047B704780B584B000AFF860B9603B605B
:102B20001346FB711CE03B68B3F1FF3F18D03B68D4
:102B3000002B07D0FEF796FA0246BB69D21A3B6813
:102B40009A420DD9FB68202283F84120FB680022BD
:102B500083F84220FB68002283F8402003230FE023
:102B6000FB681B689A69BB681A40BB689A420CBF35
:102B700001230023DBB21A46FB799A42D3D000230B
:102B800018461037BD4680BD80B584B000AFF860F0
:102B9000B9607A602CE07A68B968F86800F070F87B
:102BA0000346002B01D001232AE0BB68B3F1FF3FAD
:102BB0001ED0BB68002B07D0FEF754FA02467B6894
:102BC000D21ABB689A4213D9FB685B6C43F02002AF
:102BD000FB685A64FB68202283F84120FB680022CE
:102BE00083F84220FB68002283F84020032307E09B
:102BF000FB681B689B6903F00203022BCBD1002307
:102C000018461037BD4680BD80B584B000AFF8606F
:102C1000B9607A6028E07A68B968F86800F030F83E
:102C20000346002B01D0012326E0BB68002B07D010
:102C3000FEF718FA02467B68D21ABB689A4213D98B
:102C4000FB685B6C43F02002FB685A64FB6820223F
:102C500083F84120FB68002283F84220FB680022B1
:102C600083F84020032307E0FB681B689B6903F09F
:102C70002003202BCFD1002318461037BD4680BD3E
:102C800080B584B000AFF860B9607A60FB681B68FB
:102C90009B6903F01003102B48D11CE0BB68B3F113
:102CA000FF3F18D0BB68002B07D0FEF7DBF90246C8
:102CB0007B68D21ABB689A420DD9FB68202283F840
:102CC0004120FB68002283F84220FB68002283F841
:102CD000402003232BE0FB681B689B6903F0200363
:102CE000202BDBD1FB681B681022DA61FB681B68B4
:102CF0002022DA61F868FFF7E9FEFB681A68FB68D2
:102D00001B6859680C4B0B405360FB6804225A64E3
:102D1000FB68202283F84120FB68002283F84220D0
:102D2000FB68002283F84020012300E000231846BE
:102D30001037BD4680BD00BF00E800FE80B485B0FE
:102D400000AFF8607B600B467B8113467B72FB68AB
:102D50001A68FB681B685968BB695B0D03F48060E7
:102D60000B4B0343DB4319407B89C3F309007B7A98
:102D70001B0403F47F0318437B681843BB690343B8
:102D80000B43536000BF1437BD465DF8047B7047AA
:102D9000FF63FF0380B483B000AF786039607B6865
:102DA00093F84130DBB2202B38D17B6893F8403068
:102DB000012B01D1022332E07B68012283F84020FD
:102DC0007B68242283F841207B681B687A6812683C
:102DD000126822F001021A607B681B687A68126828
:102DE000126822F480521A607B681B687A68126845
:102DF00011683A680A431A607B681B687A6812682F
:102E0000126842F001021A607B68202283F8412098
:102E10007B68002283F84020002300E0022318464C
:102E20000C37BD465DF8047B704780B485B000AFB9
:102E3000786039600023FB607B6893F84130DBB237
:102E4000202B39D17B6893F84030012B01D102232C
:102E500033E07B68012283F840207B68242283F8DA
:102E600041207B681B687A681268126822F00102B0
:102E70001A607B681B681B68FB60FB6823F4706347
:102E8000FB603B681B02FA681343FB607B681B68AE
:102E9000FA681A607B681B687A681268126842F0E8
:102EA00001021A607B68202283F841207B6800229F
:102EB00083F84020002300E0022318461437BD4663
:102EC0005DF8047B7047000080B5ADF5007D00AF74
:102ED0003B1D18603B1D1B68002B02D1012300F035
:102EE000DABE3B1D1B681B6803F00103002B00F0DA
:102EF0006E81B54B5B6803F00C03042B0CD0B24B16
:102F00005B6803F00C03082B5AD1AF4B5B6803F4EA
:102F10008033B3F5803F53D14FF40033C7F8F43119
:102F2000D7F8F43193FAA3F3C7F8F031D7F8F031BA
:102F3000B3FA83F3DBB25B09DBB243F00103DBB22C
:102F4000012B02D1A04B1B6815E04FF40033C7F8EA
:102F5000EC31D7F8EC3193FAA3F3C7F8E8314FF42A
:102F60000033C7F8E431D7F8E43193FAA3F3C7F894
:102F7000E031954B5B6A4FF40032C7F8DC21D7F89B
:102F8000DC2192FAA2F2C7F8D821D7F8D821B2FAF8
:102F900082F252B242F0200252B2D2B202F01F02CA
:102FA000012101FA02F21340002B00F00F813B1DBA
:102FB0001B685B68002B40F00981012300F06BBEA9
:102FC0003B1D1B685B68B3F5803F06D17E4A7E4B94
:102FD0001B6843F48033136030E03B1D1B685B6863
:102FE000002B0CD1784A784B1B6823F48033136094
:102FF000754A754B1B6823F4802313601EE03B1D4C
:103000001B685B68B3F5A02F0CD16F4A6E4B1B6831
:1030100043F4802313606C4A6B4B1B6843F480338A
:1030200013600BE0684A684B1B6823F4803313601D
:10303000654A654B1B6823F4802313606249624B29
:10304000DB6A23F00F023B1D1B689B681343CB62B6
:103050003B1D1B685B68002B5AD0FEF703F8C7F8CE
:10306000F8010AE0FDF7FEFF0246D7F8F831D31A5F
:10307000642B02D9032300F00EBE4FF40033C7F8CF
:10308000D431D7F8D43193FAA3F3C7F8D031D7F8B5
:10309000D031B3FA83F3DBB25B09DBB243F0010357
:1030A000DBB2012B02D1484B1B6815E04FF4003313
:1030B000C7F8CC31D7F8CC3193FAA3F3C7F8C831AD
:1030C0004FF40033C7F8C431D7F8C43193FAA3F3EF
:1030D000C7F8C0313C4B5B6A4FF40032C7F8BC21E3
:1030E000D7F8BC2192FAA2F2C7F8B821D7F8B821D4
:1030F000B2FA82F252B242F0200252B2D2B202F0DE
:103100001F02012101FA02F21340002BAAD05EE057
:10311000FDF7A8FFC7F8F8010AE0FDF7A3FF024694
:10312000D7F8F831D31A642B02D9032300F0B3BDCA
:103130004FF40033C7F8B431D7F8B43193FAA3F39E
:10314000C7F8B031D7F8B031B3FA83F3DBB25B091B
:10315000DBB243F00103DBB2012B02D11A4B1B6837
:1031600015E04FF40033C7F8AC31D7F8AC3193FA1F
:10317000A3F3C7F8A8314FF40033C7F8A431D7F848
:10318000A43193FAA3F3C7F8A0310F4B5B6A4FF455
:103190000032C7F89C21D7F89C2192FAA2F2C7F816
:1031A0009821D7F89821B2FA82F252B242F0200266
:1031B00052B2D2B202F01F02012101FA02F2134010
:1031C000002BAAD103E000BF0010024000BF3B1D4E
:1031D0001B681B6803F00203002B00F07081D04BCA
:1031E0005B6803F00C03002B0BD0CD4B5B6803F046
:1031F0000C03082B6DD1CA4B5B6803F48033002BA2
:1032000067D10223C7F89431D7F8943193FAA3F326
:10321000C7F89031D7F89031B3FA83F3DBB25B098A
:10322000DBB243F00103DBB2012B02D1BC4B1B68C4
:1032300013E00223C7F88C31D7F88C3193FAA3F34B
:10324000C7F888310223C7F88431D7F8843193FA5C
:10325000A3F3C7F88031B24B5B6A0222C7F87C2126
:10326000D7F87C2192FAA2F2C7F87821D7F8782112
:10327000B2FA82F252B242F0200252B2D2B202F05C
:103280001F02012101FA02F21340002B07D03B1D5F
:103290001B681B69012B02D0012300F0FCBCA04875
:1032A0009F4B1B6823F0F8023B1D1B685969F823EC
:1032B000C7F87431D7F8743193FAA3F3C7F87031B3
:1032C000D7F87031B3FA83F301FA03F313430360C1
:1032D000F5E03B1D1B681B69002B00F08580012376
:1032E000C7F86C31D7F86C3193FAA3F3C7F868319B
:1032F000D7F86831B3FA83F303F1845303F58413E9
:103300009B001A4601231360FDF7ACFEC7F8F801D5
:103310000AE0FDF7A7FE0246D7F8F831D31A022BD0
:1033200002D9032300F0B7BC0223C7F86431D7F8F1
:10333000643193FAA3F3C7F86031D7F86031B3FA78
:1033400083F3DBB25B09DBB243F00103DBB2012B99
:1033500002D1734B1B6813E00223C7F85C31D7F826
:103360005C3193FAA3F3C7F858310223C7F85431FC
:10337000D7F8543193FAA3F3C7F85031684B5B6A1E
:103380000222C7F84C21D7F84C2192FAA2F2C7F8D2
:103390004821D7F84821B2FA82F252B242F0200214
:1033A00052B2D2B202F01F02012101FA02F213401E
:1033B000002BAED05A485A4B1B6823F0F8023B1D35
:1033C0001B685969F823C7F84431D7F8443193FA98
:1033D000A3F3C7F84031D7F84031B3FA83F301FAC9
:1033E00003F3134303606AE00123C7F83C31D7F8C5
:1033F0003C3193FAA3F3C7F83831D7F83831B3FA30
:1034000083F303F1845303F584139B001A460023CE
:103410001360FDF727FEC7F8F8010AE0FDF722FE6A
:103420000246D7F8F831D31A022B02D9032300F051
:1034300032BC0223C7F83431D7F8343193FAA3F3FE
:10344000C7F83031D7F83031B3FA83F3DBB25B0918
:10345000DBB243F00103DBB2012B02D1304B1B681E
:1034600013E00223C7F82C31D7F82C3193FAA3F3D9
:10347000C7F828310223C7F82431D7F8243193FA4A
:10348000A3F3C7F82031264B5B6A0222C7F81C2140
:10349000D7F81C2192FAA2F2C7F81821D7F8182100
:1034A000B2FA82F252B242F0200252B2D2B202F02A
:1034B0001F02012101FA02F21340002BAED13B1D85
:1034C0001B681B6803F00803002B00F0D8803B1D2D
:1034D0001B689B69002B67D00123C7F81431D7F80C
:1034E000143193FAA3F3C7F81031D7F81031B3FAB7
:1034F00083F31A460B4B13449B001A4601231360B7
:10350000FDF7B0FDC7F8F8010EE0FDF7ABFD024690
:10351000D7F8F831D31A022B06D90323BBE300BF37
:1035200000100240208190100223C7F80C31D7F818
:103530000C3193FAA3F3C7F808310223C7F804311A
:10354000D7F8043193FAA3F207F580731A6007F1F4
:10355000FC0302221A6007F1FC031B6893FAA3F232
:1035600007F1F8031A60A54B5A6A07F1F403022128
:10357000196007F1F4031B6893FAA3F107F1F00354
:10358000196007F1F0031B68B3FA83F35BB243F0F1
:1035900060035BB2DBB203F01F03012101FA03F306
:1035A0001340002BB1D06AE007F1EC0301221A604E
:1035B00007F1EC031B6893FAA3F207F1E8031A6022
:1035C00007F1E8031B68B3FA83F31A468C4B1344E4
:1035D0009B001A4600231360FDF744FDC7F8F8016D
:1035E00009E0FDF73FFD0246D7F8F831D31A022B68
:1035F00001D903234FE307F1E40302221A6007F124
:10360000E4031B6893FAA3F207F1E0031A6007F1E1
:10361000DC0302221A6007F1DC031B6893FAA3F2B1
:1036200007F1D8031A6007F1D40302221A6007F1E8
:10363000D4031B6893FAA3F207F1D0031A606F4B0F
:103640005A6A07F1CC030221196007F1CC031B6809
:1036500093FAA3F107F1C803196007F1C8031B68C7
:10366000B3FA83F35BB243F060035BB2DBB203F007
:103670001F03012101FA03F31340002BB1D13B1DBD
:103680001B681B6803F00403002B00F05981002322
:1036900087F8FF31594BDB6903F08053002B12D1BF
:1036A000564A564BDB6943F08053D361534BDB6979
:1036B00003F0805207F10C031A6007F10C031B683A
:1036C000012387F8FF314F4B1B6803F48073002BF5
:1036D0001AD14C4A4B4B1B6843F480731360FDF7BF
:1036E000C1FCC7F8F80109E0FDF7BCFC0246D7F8B9
:1036F000F831D31A642B01D90323CCE2414B1B6868
:1037000003F48073002BEFD03B1D1B68DB68012B9B
:1037100006D13A4A394B1B6A43F0010313622FE08A
:103720003B1D1B68DB68002B0CD1344A334B1B6AF2
:1037300023F001031362314A304B1B6A23F0040368
:1037400013621DE03B1D1B68DB68052B0CD12B4A67
:103750002A4B1B6A43F004031362284A274B1B6A57
:1037600043F0010313620BE0244A244B1B6A23F04D
:1037700001031362214A214B1B6A23F004031362E5
:103780003B1D1B68DB68002B6BD0FDF76BFCC7F89B
:10379000F8010BE0FDF766FC0246D7F8F831D31AC2
:1037A00041F28832934201D9032374E207F1C40342
:1037B00002221A6007F1C4031B6893FAA3F207F10F
:1037C000C0031A6007F1BC0302221A6007F1BC03B0
:1037D0001B6893FAA3F207F1B8031A6007F1B80364
:1037E0001B68B3FA83F3DBB25B09DBB243F002037D
:1037F000DBB2022B08D1014B1B6A13E00010024020
:10380000208190100070004007F1B40302221A607A
:1038100007F1B4031B6893FAA3F207F1B0031A602F
:10382000BB4B5B6A07F1AC020221116007F1AC02ED
:10383000126892FAA2F107F1A802116007F1A8023A
:103840001268B2FA82F252B242F0400252B2D2B2DE
:1038500002F01F02012101FA02F21340002B99D05D
:1038600064E0FDF7FFFBC7F8F8010BE0FDF7FAFB9A
:103870000246D7F8F831D31A41F28832934201D97F
:10388000032308E207F1A40302221A6007F1A4034C
:103890001B6893FAA3F207F1A0031A6007F19C03D7
:1038A00002221A6007F19C031B6893FAA3F207F146
:1038B00098031A6007F198031B68B3FA83F3DBB22D
:1038C0005B09DBB243F00203DBB2022B02D1904B67
:1038D0001B6A0DE007F1940302221A6007F19403BA
:1038E0001B6893FAA3F207F190031A60884B5B6A96
:1038F00007F18C020221116007F18C02126892FA22
:10390000A2F107F18802116007F188021268B2FA89
:1039100082F252B242F0400252B2D2B202F01F0220
:10392000012101FA02F21340002B9FD197F8FF31D9
:10393000012B05D1764A764BDB6923F08053D361A6
:103940003B1D1B68DB69002B00F0A481704B5B689A
:1039500003F00C03082B00F09B813B1D1B68DB6907
:10396000022B40F0138107F184034FF080721A603C
:1039700007F184031B6893FAA3F207F180031A602E
:1039800007F180031B68B3FA83F303F1845303F553
:1039900084139B001A4600231360FDF763FBC7F8EE
:1039A000F80109E0FDF75EFB0246D7F8F831D31ABB
:1039B000022B01D903236EE107F17C034FF0007263
:1039C0001A6007F17C031B6893FAA3F207F17803EE
:1039D0001A6007F178031B68B3FA83F3DBB25B0963
:1039E000DBB243F00103DBB2012B02D1484B1B6871
:1039F0001BE007F174034FF000721A6007F17403C3
:103A00001B6893FAA3F207F170031A6007F16C03C5
:103A10004FF000721A6007F16C031B6893FAA3F26F
:103A200007F168031A603A4B5B6A07F164024FF0D2
:103A30000071116007F16402126892FAA2F107F1B5
:103A40006002116007F160021268B2FA82F252B2AB
:103A500042F0200252B2D2B202F01F02012101FA5A
:103A600002F21340002B9DD12948294B5B6823F4B7
:103A700074123B1D1B68596A3B1D1B681B6A0B4374
:103A80001343436007F15C034FF080721A6007F143
:103A90005C031B6893FAA3F207F158031A6007F15D
:103AA00058031B68B3FA83F303F1845303F58413BB
:103AB0009B001A4601231360FDF7D4FAC7F8F801FA
:103AC00009E0FDF7CFFA0246D7F8F831D31A022BF6
:103AD00001D90323DFE007F154034FF000721A60AD
:103AE00007F154031B6893FAA3F207F150031A601D
:103AF00007F150031B68B3FA83F3DBB25B09DBB257
:103B000043F00103DBB2012B04D1014B1B681DE024
:103B10000010024007F14C034FF000721A6007F1E9
:103B20004C031B6893FAA3F207F148031A6007F1EC
:103B300044034FF000721A6007F144031B6893FAC4
:103B4000A3F207F140031A60554B5B6A07F13C0290
:103B50004FF00071116007F13C02126892FAA2F175
:103B600007F13802116007F138021268B2FA82F2E6
:103B700052B242F0200252B2D2B202F01F02012130
:103B800001FA02F21340002B9BD083E007F13403CB
:103B90004FF080721A6007F134031B6893FAA3F2A6
:103BA00007F130031A6007F130031B68B3FA83F39F
:103BB00003F1845303F584139B001A46002313601A
:103BC000FDF750FAC7F8F80109E0FDF74BFA024695
:103BD000D7F8F831D31A022B01D903235BE007F1A0
:103BE0002C034FF000721A6007F12C031B6893FA44
:103BF000A3F207F128031A6007F128031B68B3FA40
:103C000083F3DBB25B09DBB243F00103DBB2012BD0
:103C100002D1234B1B681BE007F124034FF0007215
:103C20001A6007F124031B6893FAA3F207F120033B
:103C30001A6007F11C034FF000721A6007F11C03B1
:103C40001B6893FAA3F207F118031A60144B5B6A1E
:103C500007F114024FF00071116007F114021268AD
:103C600092FAA2F107F11002116007F11002126836
:103C7000B2FA82F252B242F0200252B2D2B202F052
:103C80001F02012101FA02F21340002B9DD101E035
:103C9000012300E00023184607F50077BD4680BDEC
:103CA0000010024080B59EB000AF786039600023FC
:103CB0007B677B68002B01D1012364E1924B1B6879
:103CC00003F007023B689A4210D28F498E4B1B6863
:103CD00023F007023B6813430B608B4B1B6803F018
:103CE00007023B689A4201D001234CE17B681B68C4
:103CF00003F00203002B08D08449844B5B6823F057
:103D0000F0027B689B6813434B607B681B6803F081
:103D10000103002B00F0DF807B685B68012B3DD145
:103D20004FF400333B673B6F93FAA3F3FB66FB6EE4
:103D3000B3FA83F3DBB25B09DBB243F00103DBB21E
:103D4000012B02D1714B1B680FE04FF40033BB66AF
:103D5000BB6E93FAA3F37B664FF400333B663B6E76
:103D600093FAA3F3FB65694B5B6A4FF40032BA65C3
:103D7000BA6D92FAA2F27A657A6DB2FA82F252B212
:103D800042F0200252B2D2B202F01F02012101FA27
:103D900002F21340002B7DD10123F4E07B685B68C5
:103DA000022B3DD14FF000733B653B6D93FAA3F3BB
:103DB000FB64FB6CB3FA83F3DBB25B09DBB243F069
:103DC0000103DBB2012B02D1504B1B680FE04FF017
:103DD0000073BB64BB6C93FAA3F37B644FF0007376
:103DE0003B643B6C93FAA3F3FB63484B5B6A4FF075
:103DF0000072BA63BA6B92FAA2F27A637A6BB2FA81
:103E000082F252B242F0200252B2D2B202F01F024B
:103E1000012101FA02F21340002B3BD10123B2E051
:103E200002233B633B6B93FAA3F3FB62FB6AB3FA97
:103E300083F3DBB25B09DBB243F00103DBB2012B9E
:103E400002D1324B1B680DE00223BB62BB6A93FABE
:103E5000A3F37B6202233B623B6A93FAA3F3FB6109
:103E60002A4B5B6A0222BA61BA6992FAA2F27A61BB
:103E70007A69B2FA82F252B242F0200252B2D2B25F
:103E800002F01F02012101FA02F21340002B01D1BE
:103E9000012378E01D491D4B5B6823F003027B681A
:103EA0005B6813434B60FDF7DDF878670AE0FDF7C8
:103EB000D9F802467B6FD31A41F28832934201D976
:103EC000032360E0114B5B6803F00C027B685B68C6
:103ED0009B009A42EBD10C4B1B6803F007023B6836
:103EE0009A4215D90849084B1B6823F007023B6822
:103EF00013430B60044B1B6803F007023B689A42B4
:103F000006D001233FE000BF002002400010024025
:103F10007B681B6803F00403002B08D01C491C4B72
:103F20005B6823F4E0627B68DB6813434B607B686B
:103F30001B6803F00803002B09D01549144B5B687C
:103F400023F460527B681B69DB0013434B6000F075
:103F500025F801460E4B5B6803F0F002F0233B614D
:103F60003B6993FAA3F3FB60FB68B3FA83F322FA8D
:103F700003F3084AD35C21FA03F3074A13600020D5
:103F8000FDF72CF8002318467837BD4680BD00BFEA
:103F900000100240A8AB00080800002080B48BB0DD
:103FA00000AF0023FB610023BB6100237B62002381
:103FB0007B6100233B62294B5B68FB61FB6903F07B
:103FC0000C03042B02D0082B03D03CE0244B3B62B3
:103FD0003CE0FB6903F470124FF47013BB60BB68E4
:103FE00093FAA3F37B607B68B3FA83F322FA03F3BB
:103FF0001C4AD35C7B61194BDB6A03F00F020F2371
:104000003B613B6993FAA3F3FB60FB68B3FA83F36C
:1040100022FA03F3144AD35CBB61FB6903F48033D7
:10402000002B08D00E4ABB69B2FBF3F37A6902FB9E
:1040300003F37B6204E07B690C4A02FB03F37B62BF
:104040007B6A3B6202E0064B3B6200BF3B6A18465C
:104050002C37BD465DF8047B704700BF001002405E
:1040600000127A0088AB000898AB000800093D00F8
:1040700080B400AF034B1B681846BD465DF8047B57
:10408000704700BF0800002080B582B000AFFFF786
:10409000EFFF01460B4B5B6803F4E0624FF4E06313
:1040A0007B607B6893FAA3F33B603B68B3FA83F3CE
:1040B00022FA03F3044AD35C21FA03F318460837C3
:1040C000BD4680BD00100240B8AB000880B582B08C
:1040D00000AFFFF7CDFF01460B4B5B6803F4605266
:1040E0004FF460537B607B6893FAA3F33B603B68BB
:1040F000B3FA83F322FA03F3044AD35C21FA03F3FD
:1041000018460837BD4680BD00100240B8AB000815
:1041100080B592B000AF786000233B640023FB635E
:104120007B681B6803F48033002B00F0CF800023F2
:1041300087F847308D4BDB6903F08053002B0ED19D
:104140008A4A8A4BDB6943F08053D361874BDB6932
:1041500003F08053BB60BB68012387F84730844B72
:104160001B6803F48073002B18D1814A804B1B68B5
:1041700043F480731360FCF775FF386408E0FCF7C4
:1041800071FF02463B6CD31A642B01D90323E9E08B
:10419000774B1B6803F48073002BF0D0734B1B6AC2
:1041A00003F44073FB63FB6B002B7CD07B685B6884
:1041B00003F44072FB6B9A4275D06C4B1B6A23F47C
:1041C0004073FB634FF480333B633B6B93FAA3F381
:1041D000FB62FB6AB3FA83F31A46664B13449B00F7
:1041E0001A46012313604FF48033BB63BB6B93FA11
:1041F000A3F37B637B6BB3FA83F31A465D4B1344E3
:104200009B001A4600231360584AFB6B1362FB6B3A
:1042100003F00103002B46D0FCF724FF38640AE0CA
:10422000FCF720FF02463B6CD31A41F288329342DE
:1042300001D9032396E00223BB62BB6A93FAA3F37E
:104240007B6202233B623B6A93FAA3F3FB61FB6947
:10425000B3FA83F3DBB25B09DBB243F00203DBB2F8
:10426000022B02D1414B1B6A07E00223BB61BB69F1
:1042700093FAA3F37B613D4B5B6A02223A613A6990
:1042800092FAA2F2FA60FA68B2FA82F252B242F0FC
:10429000400252B2D2B202F01F02012101FA02F230
:1042A0001340002BBCD03149304B1B6A23F44072C1
:1042B0007B685B6813430B6297F84730012B05D18D
:1042C0002A4A2A4BDB6923F08053D3617B681B6841
:1042D00003F00103002B08D02449244B1B6B23F06F
:1042E00003027B689B6813430B637B681B6803F0C6
:1042F0002003002B08D01D491C4B1B6B23F0100220
:104300007B68DB6813430B637B681B6803F08003E7
:10431000002B08D01549154BDB6A23F4F8727B6833
:104320001B691343CB627B681B6803F48053002B2B
:1043300008D00E490D4B1B6B23F480727B685B69C0
:1043400013430B637B681B6803F48043002B08D086
:104350000649064B1B6B23F480527B689B69134311
:104360000B63002318464837BD4680BD001002404D
:10437000007000400081901080B582B000AF78607E
:104380007B68002B01D1012343E07B6893F86930FF
:10439000DBB2002B06D17B68002283F868207868A6
:1043A00004F0C8FC7B68242283F869207B681B68C2
:1043B0007A681268126822F001021A60786800F0C8
:1043C00081FA0346012B01D1012322E07B685B6A5D
:1043D000002B02D0786800F0DBFB7B681B687A68F2
:1043E0001268526822F490425A607B681B687A68AF
:1043F0001268926822F02A029A607B681B687A68C9
:104400001268126842F001021A60786800F062FCDB
:10441000034618460837BD4680BD80B588B002AF58
:10442000F860B9603B601346FB8000237B61FB684A
:1044300093F86930DBB2202B77D1BB68002B02D018
:10444000FB88002B01D1012370E0FB6893F86830F2
:10445000012B01D1022369E0FB68012283F8682067
:10446000FB680022DA66FB68212283F86920FCF7EA
:10447000F9FD7861FB68FA88A3F85020FB68FA8898
:10448000A3F8522034E0FB68B3F852309BB2013BF2
:104490009AB2FB68A3F852203B6800937B69002224
:1044A0008021F86800F05FFC0346002B01D0032355
:1044B0003CE0FB689B68B3F5805F11D1FB681B692A
:1044C000002B0DD1BB683B61FB681B683A69128801
:1044D000C2F3080292B21A85BB680233BB6007E0E0
:1044E000FB681A68BB68591CB9601B789BB21385BE
:1044F000FB68B3F852309BB2002BC4D13B680093E9
:104500007B6900224021F86800F02DFC0346002B57
:1045100001D003230AE0FB68202283F86920FB68AE
:10452000002283F86820002300E002231846183791
:10453000BD4680BD80B485B000AFF860B960134659
:10454000FB80FB6893F86A30DBB2202B72D1BB682A
:10455000002B02D0FB88002B01D101236BE0FB680C
:1045600093F86830012B01D1022364E0FB6801223B
:1045700083F86820FB68BA685A65FB68FA88A3F874
:104580005820FB68FA88A3F85A20FB689B68B3F5AB
:10459000805F0ED1FB681B69002B05D1FB6840F2E0
:1045A000FF12A3F85C2028E0FB68FF22A3F85C2040
:1045B00023E0FB689B68002B0DD1FB681B69002B77
:1045C00004D1FB68FF22A3F85C2016E0FB687F2281
:1045D000A3F85C2011E0FB689B68B3F1805F0CD10D
:1045E000FB681B69002B04D1FB687F22A3F85C20C9
:1045F00003E0FB683F22A3F85C20FB680022DA6638
:10460000FB68222283F86A20FB68002283F8682076
:10461000FB681B68FA681268926842F001029A60AF
:10462000FB681B68FA681268126842F490721A609C
:10463000002300E0022318461437BD465DF8047BD2
:104640007047000080B586B000AF78607B681B685B
:10465000DB697B617B681B681B683B617B6903F0DE
:104660000F03FB60FB68002B0DD17B6903F0200377
:10467000002B08D03B6903F02003002B03D078689F
:1046800000F05FFCFAE07B681B689B68BB60FB681E
:10469000002B00F0BA80BB6803F00103002B05D1AA
:1046A0003B6903F49073002B00F0AF807B6903F04B
:1046B0000103002B0ED03B6903F48073002B09D05B
:1046C0007B681B6801221A627B68DB6E43F0010283
:1046D0007B68DA667B6903F00203002B0ED0BB68AF
:1046E00003F00103002B09D07B681B6802221A62C9
:1046F0007B68DB6E43F004027B68DA667B6903F05B
:104700000403002B0ED0BB6803F00103002B09D07B
:104710007B681B6804221A627B68DB6E43F002022E
:104720007B68DA667B6903F00803002B13D03B69D2
:1047300003F02003002B04D1BB6803F00103002B1E
:1047400009D07B681B6808221A627B68DB6E43F025
:1047500008027B68DA667B68DB6E002B00F08D80D8
:104760007B6903F02003002B07D03B6903F0200393
:10477000002B02D0786800F0E4FB7B68DB6E03F06E
:104780000803002B06D17B681B689B6803F040037D
:10479000402B31D1786800F030FB7B681B689B6848
:1047A00003F04003402B23D17B681B687A681268B2
:1047B000926822F040029A607B685B6E002B13D0F7
:1047C0007B685B6E2F4A5A637B685B6E1846FDF709
:1047D00016FC0346002B16D07B685B6E5B6B7A6819
:1047E000526E104698470EE0786800F061F80AE0D3
:1047F000786800F05DF806E0786800F059F87B68AA
:104800000022DA6639E000BF37E07B6903F48013E9
:10481000002B15D0BB6803F48003002B10D07B68FD
:104820001B684FF480121A627B68202283F869208B
:104830007B68202283F86A20786800F0ECFB1DE09A
:104840007B6903F08003002B08D03B6903F08003F1
:10485000002B03D0786800F004FB0FE07B6903F0C5
:104860004003002B0AD03B6903F04003002B05D026
:10487000786800F04EFB00BF00E000BF1837BD466F
:1048800080BD00BF374E000880B483B000AF7860B1
:1048900000BF0C37BD465DF8047B704780B483B021
:1048A00000AF786000BF0C37BD465DF8047B7047F1
:1048B00080B483B000AF786000BF0C37BD465DF8B0
:1048C000047B704790B587B000AF78600023FB6031
:1048D0001023FB7500237B810023BB820023FB7424
:1048E0007B689A687B681B691A437B685B691A431B
:1048F0007B68DB691343FB607B681A687B681B6815
:1049000019689E4B0B40F9680B4313607B681B686A
:104910007A681268526822F440517A68D2680A4371
:104920005A607B689A697B681B6A1343FB607B68EB
:104930001B687A681268926822F43061FA680A4348
:104940009A607B681B688E4A934221D18D4B1B6B0A
:1049500003F00303032B17D801A252F823F000BF82
:10496000714900087D49000883490008774900081B
:104970000023FB751EE00223FB751BE00423FB757F
:1049800018E00823FB7515E01023FB7500BF11E04C
:104990007B681B687C4A934202D10023FB7509E0C7
:1049A0007B681B68794A934202D10023FB7501E0C2
:1049B0001023FB757B68DB69B3F5004F6FD1FB7D7E
:1049C000082B57D801A252F823F000BFF149000884
:1049D0000D4A0008294A0008754A0008434A0008A1
:1049E000754A0008754A0008754A00085F4A0008C1
:1049F000FFF74AFB03465A007B685B685B081A4472
:104A00007B685B68B2FBF3F3BB8236E0FFF75EFBCB
:104A100003465A007B685B685B081A447B685B68E6
:104A2000B2FBF3F3BB8228E07B685B685B0803F5AD
:104A3000740303F510537A685268B3FBF2F3BB8238
:104A40001BE0FFF7ABFA03465A007B685B685B0824
:104A50001A447B685B68B2FBF3F3BB820DE07B68B2
:104A60005B685B0803F580327B685B68B2FBF3F33D
:104A7000BB8202E00123FB7400BFBB8A23F00F035B
:104A80007B81BB8A5B109BB203F007039AB27B89E0
:104A900013437B817B681B687A89DA6069E0FB7D60
:104AA000082B63D801A252F823F000BFD14A0008B6
:104AB000F14A0008114B00086D4B0008314B00080B
:104AC0006D4B00086D4B00086D4B0008514B000802
:104AD0007B681C68FFF7D8FA02467B685B685B0856
:104AE0001A447B685B68B2FBF3F39BB2E36040E07F
:104AF0007B681C68FFF7EAFA02467B685B685B0824
:104B00001A447B685B68B2FBF3F39BB2E36030E06E
:104B10007B681A687B685B685B0803F5F40303F540
:104B2000905379684968B3FBF1F39BB2D36020E0FE
:104B30007B681C68FFF732FA02467B685B685B089B
:104B40001A447B685B68B2FBF3F39BB2E36010E04E
:104B50007B681B687A685268520802F500417A68DF
:104B60005268B1FBF2F292B2DA6002E00123FB7408
:104B700000BFFB7C18461C37BD4690BDF369FFEFB4
:104B8000003801400010024000440040004800404E
:104B900080B483B000AF78607B685B6A03F0010388
:104BA000002B0AD07B681B687A681268526822F46E
:104BB00000317A68926A0A435A607B685B6A03F044
:104BC0000203002B0AD07B681B687A68126852685F
:104BD00022F480317A68D26A0A435A607B685B6A41
:104BE00003F00403002B0AD07B681B687A68126804
:104BF000526822F480217A68126B0A435A607B68FB
:104C00005B6A03F00803002B0AD07B681B687A6894
:104C10001268526822F400417A68526B0A435A6063
:104C20007B685B6A03F01003002B0AD07B681B686B
:104C30007A681268926822F480517A68926B0A430B
:104C40009A607B685B6A03F02003002B0AD07B68C4
:104C50001B687A681268926822F400517A68D26BF5
:104C60000A439A607B685B6A03F04003002B1AD00A
:104C70007B681B687A681268526822F480117A682F
:104C8000126C0A435A607B681B6CB3F5801F0AD113
:104C90007B681B687A681268526822F4C0017A68DF
:104CA000526C0A435A607B685B6A03F08003002BF6
:104CB0000AD07B681B687A681268526822F4002167
:104CC0007A68926C0A435A6000BF0C37BD465DF8A3
:104CD000047B704780B586B002AF78600023FB602C
:104CE0007B680022DA66FCF7BDF9F8607B681B6818
:104CF0001B6803F00803082B0ED16FF07E4300936E
:104D0000FB6800224FF40011786800F02CF803468D
:104D1000002B01D0032322E07B681B681B6803F093
:104D20000403042B0ED16FF07E430093FB68002236
:104D30004FF48001786800F016F80346002B01D08C
:104D400003230CE07B68202283F869207B68202203
:104D500083F86A207B68002283F8682000231846C5
:104D60001037BD4680BD80B584B000AFF860B96033
:104D70003B601346FB712CE0BB69B3F1FF3F28D0C9
:104D8000BB69002B07D0FCF76DF902463B68D21ACD
:104D9000BB699A421DD9FB681B68FA6812681268E1
:104DA00022F4D0721A60FB681B68FA681268926875
:104DB00022F001029A60FB68202283F86920FB68D8
:104DC000202283F86A20FB68002283F868200323EE
:104DD0000FE0FB681B68DA69BB681A40BB689A423F
:104DE0000CBF01230023DBB21A46FB799A42C3D0E1
:104DF000002318461037BD4680BD80B483B000AF95
:104E000078607B681B687A681268126822F4907276
:104E10001A607B681B687A681268926822F0010247
:104E20009A607B68202283F86A2000BF0C37BD4659
:104E30005DF8047B704780B584B000AF78607B6814
:104E40005B6AFB60FB680022A3F85A20FB68002223
:104E5000A3F85220F868FFF72BFD00BF1037BD46BE
:104E600080BD80B485B000AF78607B6893F869300E
:104E7000DBB2212B46D17B68B3F852309BB2002BBA
:104E800011D17B681B687A681268126822F0800270
:104E90001A607B681B687A681268126842F04002E8
:104EA0001A6000232FE07B689B68B3F5805F14D104
:104EB0007B681B69002B10D17B68DB6CFB607B6817
:104EC0001B68FA681288C2F3080292B21A857B68DE
:104ED000DB6C9A1C7B68DA6409E07B681A687B6883
:104EE000DB6C581C7968C8641B789BB213857B689F
:104EF000B3F852309BB2013B9AB27B68A3F85220C0
:104F0000002300E0022318461437BD465DF8047BF9
:104F1000704780B582B000AF78607B681B687A68A4
:104F20001268126822F040021A607B68202283F81F
:104F300069207868FFF7A8FC002318460837BD46AB
:104F400080BD80B584B000AF78607B68B3F85C301A
:104F5000FB817B6893F86A30DBB2222B4ED17B68F1
:104F60001B689B8CBB817B689B68B3F5805F12D10B
:104F70007B681B69002B0ED17B685B6DBB60BA89B7
:104F8000FB8913409AB2BB681A807B685B6D9A1CE0
:104F90007B685A650BE07B685B6D591C7A685165CC
:104FA000BA89D1B2FA89D2B20A40D2B21A707B68F9
:104FB000B3F85A309BB2013B9BB27A681946A2F80B
:104FC0005A10002B18D17B681B687A681268126827
:104FD00022F490721A607B681B687A681268926883
:104FE00022F001029A607B68202283F86A207868A8
:104FF000FFF754FC00230AE0002308E07B681B68ED
:105000007A681268926942F008029A61022318468F
:105010001037BD4680BD80B483B000AF786000BF5C
:105020000C37BD465DF8047B7047000000000000AF
:10503000B0B584B000AF786039604FF00003FB601A
:105040003B68073B7A6813441B78A3F13002134690
:105050009B0013445B0019463B68063B7A68134487
:105060001B78303B0B441846FBF754FA04460D46B8
:105070003B68043B7A6813441B78303B1846FBF7C7
:1050800049FA57A3D3E90023FBF7AAFA02460B46D5
:1050900020462946FBF7F2F803460C4625461C46F7
:1050A0003B68033B7A6813441B78303B1846FBF798
:1050B00031FA4DA3D3E90023FBF792FA02460B46DF
:1050C00020462946FBF7DAF803460C4625461C46DF
:1050D0003B68023B7A6813441B78303B1846FBF769
:1050E00019FA43A3D3E90023FBF77AFA02460B46E9
:1050F00020462946FBF7C2F803460C4625461C46C7
:105100003B68013B7A6813441B78303B1846FBF739
:1051100001FA39A3D3E90023FBF762FA02460B46F2
:1051200020462946FBF7AAF803460C4618462146B6
:10513000FBF72EFD0346FB603B68083B7A6813448F
:105140001B78303B07EE903AB8EEE77AD7ED036A6A
:105150009FED216AC6EE867A77EE277AC7ED037A4D
:105160003B68082B14DD3B68093B7A6813441B78C5
:10517000A3F1300213469B0013445B0007EE903A04
:10518000F8EEE77A97ED037A77EE277AC7ED037AA0
:105190003B68092B15DD3B680A3B7A6813441B7892
:1051A000303B642202FB03F307EE903AF8EEE77A15
:1051B00097ED037A77EE277AC7ED037A074AFB6803
:1051C0001360FB6807EE903AB0EE670A1037BD46F1
:1051D000B0BD00BFAFF3008000007042A800002007
:1051E0009A9999999999B93F7B14AE47E17A843F8E
:1051F000FCA9F1D24D62503F2D431CEBE2361A3F21
:10520000B0B588B000AFF860B96087ED010A134609
:10521000FB700023FB610023BB617868FBF78CF90E
:1052200003460C4644EC103B04F042FB54EC103BAC
:1052300018462146FBF784FC0346FB617868FBF7C0
:105240007BF904460D467868FBF776F902460B4673
:1052500043EC102B04F02CFB53EC102B204629467A
:10526000FBF70AF803460C46184621463DA3D3E94E
:105270000023FBF7B5F903460C4644EC173BB0EEB0
:10528000470AF0EE670A04F013FB54EC103B184693
:105290002146FBF755FC0346BB6101237B6120E0FF
:1052A000BA687B69D31A1A46FB689818BA692C4BFE
:1052B00083FB02139910D317C91A0B469B000B44AA
:1052C0005B00D11ACBB23033DBB20370BB69244A26
:1052D00082FB03129210DB17D31ABB617B69013387
:1052E0007B617B69062BDBDDBB68073BFA681344F7
:1052F0002E221A7008237B6120E0BA687B69D31ADA
:105300001A46FB689818FA69154B83FB021399102B
:10531000D317C91A0B469B000B445B00D11ACBB2C2
:105320003033DBB20370FB690D4A82FB031292102B
:10533000DB17D31AFB617B6901337B61FB69002BAF
:10534000DBDCBA687B69D31A1A46FB681344FA7827
:105350001A7000BF2037BD46B0BD00BFAFF300805C
:10536000676666660000000080842E4180B485B0C8
:1053700000AF0346FB710023FB60FB792F2B06D99E
:10538000FB79392B03D8FB79303BFB6008E0FB79D4
:10539000402B05D9FB79462B02D8FB79373BFB60C4
:1053A000FB6818461437BD465DF8047B7047000063
:1053B0002DE9B0438AB000AFF860B9607A6000238D
:1053C000FB610AE0FB69FA6813441B782E2B01D1BC
:1053D000FB697B62FB690133FB61FA69BB689A4236
:1053E000F0DB4FF00003BB617B6A0133FB6133E00C
:1053F000B869FBF7A1F804460D46FA697B6AD31A2F
:105400001846FBF787F802460B4643EC112B9FED3D
:10541000660B04F017FB59EC108BFB69FA68134418
:105420001B78303B1846FBF775F802460B464046A2
:105430004946FBF7D5F802460B4620462946FAF7BF
:105440001DFF03460C4618462146FBF7A1FB034609
:10545000BB61FB690133FB61FA69BB689A42C7DB38
:105460007B6A013BFB6134E0B869FBF765F80446F1
:105470000D467B6A5A1EFB69D31A1846FBF74AF899
:1054800002460B4643EC112B9FED490B04F0DAFA70
:1054900059EC108BFB69FA6813441B78303B1846B3
:1054A000FBF738F802460B4640464946FBF798F8AA
:1054B00002460B4620462946FAF7E0FE03460C4614
:1054C00018462146FBF764FB0346BB61FB69013BC1
:1054D000FB61FB69002BC7DA374ABB691360D7ED64
:1054E000067AB2EE047A67EE877AC7ED067AB86973
:1054F000FBF722F803460C4644EC103B04F05CFA40
:1055000054EC103B18462146FBF71AFB03467B611F
:1055100000233B620623FB613CE0FB69052B05D1C0
:10552000FB697A6813442E221A7030E07B69002BE5
:105530001DDDFB697A68D0187A69204B83FB021362
:105540009910D317C91A0B469B000B445B00D11A64
:10555000CBB23033DBB203707B69184A82FB031293
:105560009210DB17D31A7B6101233B6204E0FB69D5
:105570007A68134420221A703B6A002B07D17B689B
:10558000043330221A707B68063330221A70FB69AC
:10559000013BFB61FB69002BBFDA00BF2837BD462A
:1055A000BDE8B083AFF300809A9999999999B93F72
:1055B0000000000000002440AC0000206766666622
:1055C00080B487B000AFF860B9607A603B600023B8
:1055D0007B6100233B61FB6824221A7000233B613E
:1055E00001237B610DE07B69FA6813443A69B9686D
:1055F0000A4412781A703B6901333B617B690133BD
:105600007B617B69082BEEDDFB6809332C221A7065
:1056100000233B610A237B610DE07B69FA68134438
:105620003A6979680A4412781A703B6901333B6120
:105630007B6901337B617B690E2BEEDDFB680F33E9
:105640002C221A7000233B6110237B610DE07B69E3
:10565000FA6813443A6939680A4412781A703B6947
:1056600001333B617B6901337B617B69172BEEDD85
:10567000FB6818332C221A7000233B6119237B61CD
:105680000DE07B69FA6813443A69396A0A44127872
:105690001A703B6901333B617B6901337B617B6934
:1056A0001B2BEEDDFB681C332C221A7000233B61A0
:1056B0001D237B610DE07B69FA6813443A69796ABE
:1056C0000A4412781A703B6901333B617B690133EC
:1056D0007B617B691F2BEEDDFB6820332C221A7067
:1056E00000233B6121237B610DE07B69FA68134451
:1056F0003A69B96A0A4412781A703B6901333B610E
:105700007B6901337B617B69232BEEDDFB682433EE
:105710002C221A7000233B6125237B610DE07B69FD
:10572000FA6813443A69F96A0A4412781A703B69B4
:1057300001333B617B6901337B617B69282BEEDDA3
:10574000FB6829332C221A7000233B612A237B61DA
:105750000DE07B69FA6813443A69396B0A441278A0
:105760001A703B6901333B617B6901337B617B6963
:105770002D2BEEDDFB682E332C221A7000233B61AB
:105780002F237B610DE07B69FA6813443A69796BDA
:105790000A4412781A703B6901333B617B6901331B
:1057A0007B617B69322BEEDDFB6833332C221A7070
:1057B00000233B6134237B610DE07B69FA6813446D
:1057C0003A69B96B0A4412781A703B6901333B613C
:1057D0007B6901337B617B693D2BEEDDFB683E33EA
:1057E0002C221A7000233B613F237B610DE07B6913
:1057F000FA6813443A69F96B0A4412781A703B69E3
:1058000001333B617B6901337B617B69492BEEDDB1
:10581000FB684A332C221A7000233B614B237B61C7
:105820000DE07B69FA6813443A69396C0A441278CE
:105830001A703B6901333B617B6901337B617B6992
:10584000512BEEDDFB6852332C221A7000233B6192
:1058500053237B610DE07B69FA6813443A69796CE4
:105860000A4412781A703B6901333B617B6901334A
:105870007B617B69552BEEDDFB6856332C221A7059
:1058800000233B6157237B610DE07B69FA68134479
:105890003A69B96C0A4412781A703B6901333B616A
:1058A0007B6901337B617B69592BEEDDFB685A33E1
:1058B0000A221A7000BF1C37BD465DF8047B704792
:1058C00090B585B000AF786087ED000AD7ED007A1B
:1058D0009FED387AF4EEC77AF1EE10FA5AD53868AF
:1058E000FAF72AFE03460C4644EC103B04F064F839
:1058F00054EC103B18462146FBF722F90346FB60A7
:105900007B68981CFA682C4B83FB02139910D31701
:10591000C91A0B469B000B445B00D11ACBB2303343
:10592000DBB20370FB68244A82FB03129210DB1780
:10593000D31AFB600123BB600123BB6026E0FB6838
:10594000002B1BDDBB687A68D018FA681A4B83FB02
:1059500002139910D317C91A0B469B000B445B0026
:10596000D11ACBB23033DBB20370FB68124A82FB30
:1059700003129210DB17D31AFB6004E0BB687A684D
:10598000134420221A70BB68013BBB60BB68002B2C
:10599000D5DA0BE07B6802332A221A707B68013368
:1059A0002A221A707B6801332A221A7000BF14372A
:1059B000BD4690BD00007A446766666690B585B0C6
:1059C00000AF786087ED000AD7ED007AB2EE047A76
:1059D000F4EEC77AF1EE10FA3CD5D7ED007AB2EECC
:1059E000047A67EE877A17EE900AFAF7A5FD034668
:1059F0000C4644EC103B03F0DFFF54EC103B184620
:105A00002146FBF79DF80346FB607B68981CFA680B
:105A1000184B83FB02139910D317C91A0B469B002E
:105A20000B445B00D11ACBB23033DBB20370FB689E
:105A3000104A82FB03129210DB17D31AFB60FB683B
:105A4000DBB23033DAB27B681A707B6801332E2206
:105A50001A700AE07B6802332A221A707B680133CD
:105A60002A221A707B682A221A7000BF1437BD469A
:105A700090BD00BF6766666680B582B002AF132036
:105A8000FBF7FCFA0123019301230093002300227A
:105A90000021002000F074F80420FBF7EFFA012346
:105AA000019301230093002300220021002000F035
:105AB00067F80123019301230093002300220021B2
:105AC000002000F05DF800230193012300930023E0
:105AD00000220021002000F053F80023019301234D
:105AE0000093002300220021002000F049F8002349
:105AF000019300230093002301220021002000F0E5
:105B00003FF800230193002300930023002200218B
:105B1000002000F035F800230193012300930123B6
:105B200001220021002000F02BF800230193002324
:105B30000093002300220021002000F021F801231F
:105B4000019300230093002300220021002000F095
:105B500017F8002301930023009300230022002163
:105B6000002000F00DF8002301930123009301238E
:105B700000220021002000F003F800BFBD4680BDD8
:105B800080B584B000AFF860B9607A603B60FB68B4
:105B9000DBB21A464FF400511F48FCF7E5FBBB6827
:105BA000DBB21A464FF480411B48FCF7DDFB0122B3
:105BB0004FF400411848FCF7D7FB7B68DBB21A466C
:105BC0004FF480511448FCF7CFFB3B68DBB21A4618
:105BD0004FF400611048FCF7C7FBBB69DBB21A4603
:105BE00004210D48FCF7C0FBFB69DBB21A46022119
:105BF0000948FCF7B9FB0120FBF740FA00224FF4FB
:105C000000410548FCF7B0FB0120FBF737FA00BF65
:105C10001037BD4680BD00BF0004004800000000F2
:105C200090B58FB002AF87ED030AB86079600023AA
:105C30000193002300930023002200210020FFF79E
:105C40009FFF0123019300230093002300220021E2
:105C50000020FFF795FF0123BB62F868FAF76CFCA0
:105C600003460C4644EC103B03F0A6FE54EC103BFC
:105C700018462146FAF764FF03467B627B6A092BCC
:105C800001DD0223BB627B6A622B01DD0323BB6261
:105C90007B6A40F2E632934201DD0423BB627B6AF9
:105CA00042F20E72934201DD0523BB620123FB62C7
:105CB00029E0BA6AFB6AD31A1846FAF72BFC0346A6
:105CC0000C4644EC113B9FED900B03F0BBFE54ECF3
:105CD000103B18462146FAF733FF0346BB617A6A48
:105CE000BB6992FBF3F37B617B6ABA6993FBF2F2C7
:105CF000B96901FB02F29B1A7B62786900F008F92E
:105D0000FB6A0133FB62FA6ABB6A9A42D1DD002367
:105D10000193012300930123002200210120FFF7BA
:105D20002FFF01230193002300930123012200216F
:105D30000120FFF725FF0023019300230093012397
:105D4000012200210020FFF71BFF01230193002304
:105D500000930023002200210020FFF711FFBB6801
:105D6000012B13D100230193002300930123002270
:105D700000210120FFF704FF00230193012300937A
:105D80000023002200210120FFF7FAFE01233B62DD
:105D90000023FB617B68002B06DA0123FB617B6833
:105DA000002BB8BF5B427B607B68092B01DD0223BF
:105DB0003B623A6AFB691344C3F147033B613B69A9
:105DC000462B13D1002301930023009301230122CA
:105DD00000210020FFF7D4FE00230193012300934C
:105DE0000123002200210020FFF7CAFE3B69452B5A
:105DF00013D10023019300230093012301220021EA
:105E00000020FFF7BDFE012301930023009301232F
:105E1000002200210020FFF7B3FE3B69442B13D181
:105E2000002301930023009301230122002100207D
:105E3000FFF7A6FE00230193002300930123002215
:105E400000210020FFF79CFEFB69012B13D10023EA
:105E50000193012300930023002200210120FFF77A
:105E60008FFE0123019300230093012301220021CF
:105E70000120FFF785FE0123FB6229E03A6AFB6AF5
:105E8000D31A1846FAF746FB03460C4644EC113B7E
:105E90009FED1D0B03F0D6FD54EC103B1846214638
:105EA000FAF74EFE0346BB617A68BB6992FBF3F3D7
:105EB0007B617B68BA6993FBF2F2B96901FB02F27C
:105EC0009B1A7B60786900F023F8FB6A0133FB6260
:105ED000FA6A3B6A9A42D1DD0023019300230093C2
:105EE0000123002200210120FFF74AFE0123019334
:105EF000012300930023002200210120FFF740FE30
:105F000000BF3437BD4690BD0000000000002440B3
:105F100080B588B002AF786001230193012300931C
:105F20000023002200210120FFF72AFE00237B61CD
:105F300000233B610023FB600023BB607B68072BD1
:105F400001DD01237B617B68042B08D07B68052B76
:105F500005D07B68062B02D07B68072B01D101237B
:105F60003B617B68022B08D07B68032B05D07B68E4
:105F7000062B02D07B68072B01D10123FB607B68D5
:105F8000002B03F00103B8BF5B42012B01D10123B9
:105F9000BB60BB680193FB6800933B697A69002191
:105FA0000120FFF7EDFD00BF1837BD4680BD0000A2
:105FB00080B500AF2E4B76225A702D4B01229A707D
:105FC0002B4B2C4A5A602A4B2B4A9A60284B2B4A5F
:105FD000DA60274800F052FB03461A46284B1A7035
:105FE000234B012283F83A20214B052283F83820E5
:105FF0001F4B022283F839201D4B042283F83B20DB
:106000001B4B002283F83C201E4B01221A701D4BB3
:106010001B7843F00203DAB21A4B1A70194B1B7843
:1060200043F00403DAB2174B1A70164B1B7843F097
:106030001003DAB2134B1A70124B1B7843F00803AB
:10604000DAB2104B1A700F4B1B780949184600F052
:1060500009FC03461A460A4B1A700549032000F052
:1060600056FC03461A46064B1A7000BF80BD00BF9F
:10607000D4000020A1600008E960000889600008E1
:10608000900000206C01002080B582B000AF7860E5
:106090007868FAF7F3FF00BF0837BD4680BD0000FF
:1060A00080B588B004AF3A601A460346FB710B46D0
:1060B000BB711346BB800023FB73BB799AB2C82324
:1060C0000293BB8801933B6800930123EC210548B0
:1060D000FCF716FB0346FB7397F90F301846103791
:1060E000BD4680BD1401002080B588B004AF3A6081
:1060F0001A460346FB710B46BB711346BB80002357
:10610000FB73BB799AB2C8230293BB8801933B68A7
:1061100000930123EC210548FCF7CCF90346FB73FF
:1061200097F90F3018461037BD4680BD1401002086
:1061300080B500AF164A1749072000F064FC0346FB
:106140001A46154B1A70134B1B685B09134AA2FBC6
:106150000323DB09124A126813441A46104B1A60D3
:106160000C4B5B680F4A82FB03125211DB17D21AE9
:106170000D4B1B6813440C4A1360064B9B689B0A2B
:106180000A4A126813441A46084B1A6000BF80BDC1
:10619000D40000206001002090000020C55A7C0A35
:1061A000B00000201F85EB51B8000020B400002093
:1061B00080B584B000AFF860B9607A603B60396840
:1061C000F86800F00DF8B969B86800F009F8F969E5
:1061D000786800F005F800BF1037BD4680BD0000AC
:1061E00080B485B000AF786039600023FB603B6805
:1061F000002B01DA0123FB603B68002BB8BF5B4238
:106200003B607B68981C3A68364B83FB02139910FD
:10621000D317C91A0B469B000B445B00D11ACBB2B3
:106220003033DBB203703B682E4A82FB03129210BC
:10623000DB17D31A3B60FB68012B20D13B68092B8D
:1062400015DD7B682D221A707B68581C3A68254B37
:1062500083FB02139910D317C91A0B469B000B44FA
:106260005B00D11ACBB23033DBB2037034E07B6811
:1062700001332D221A707B6820221A702CE0012332
:10628000BB6026E03B68002B1BDDBB687A68D0183A
:106290003A68144B83FB02139910D317C91A0B46A3
:1062A0009B000B445B00D11ACBB23033DBB20370DE
:1062B0003B680C4A82FB03129210DB17D31A3B6037
:1062C00004E0BB687A68134420221A70BB68013B63
:1062D000BB60BB68002BD5DA00BF1437BD465DF844
:1062E000047B70476766666680B500AF164B174A39
:1062F0001A60154B164A5A60134B164A9A6000F002
:1063000063F91549104801F0F6FC0246134B1A6078
:10631000124B1B68002B00D0FEE701210A4801F058
:106320009AFC0421084801F04AFC0021064801F0CB
:106330006CFC0321044801F0C7FB0021024801F076
:10634000E9FB00BF80BD00BF74010020D9650008D3
:10635000296600081401002080010020840100202B
:1063600080B500AF19491A4801F09BFC174B1B7808
:10637000002B29D006220021164802F071FE154993
:10638000134801F0A7FC134BB3F90030184601F095
:1063900083FBF0EE407A104BC3ED007A0D4BB3F95E
:1063A0000230184601F078FBF0EE407A0B4BC3ED5B
:1063B000007A084BB3F90430184601F06DFBF0EE9B
:1063C000407A074BC3ED007A00BF80BD700100200A
:1063D00074010020940000209C000020A0000020F8
:1063E000A4000020B0B588B000AFF860B9607A6052
:1063F0003B60394B1B681846FAF79EF802460B467D
:1064000043EC102B03F0D8FA53EC102B144683F016
:10641000004520462946FAF793FB0346FB612F4BC4
:106420001B681846FAF788F803460C4644EC103B04
:1064300003F0C2FA54EC103B18462146FAF780FBF1
:106440000346BB61264B1B681846FAF775F80346EE
:106450000C4644EC103B03F0AFFA54EC103B1846EA
:106460002146FAF76DFB03467B61FB69B3F57A7F42
:1064700002DB40F2E733FB61FB6913F57A7F01DC55
:10648000184BFB61BB69B3F57A7F02DB40F2E7335F
:10649000BB61BB6913F57A7F01DC124BBB617B6981
:1064A000B3F57A7F02DB40F2E7337B617B6913F55A
:1064B0007A7F01DC0B4B7B61F969F86800F014F816
:1064C000B969B86800F010F87969786800F00CF8DC
:1064D00000BF2037BD46B0BD9C000020A0000020BA
:1064E000A400002019FCFFFF80B487B000AF7860E3
:1064F000396000237B610023FB603B68002B01DADD
:1065000001237B613B68002BB8BF5B423B607B682B
:10651000D81C3A682B4B83FB02139910D317C91A66
:106520000B469B000B445B00D11ACBB23033DBB27D
:1065300003703B68234A82FB03129210DB17D31AC5
:106540003B6002233B6134E03B68002B1BDD3B6971
:106550007A68D0183A681B4B83FB02139910D31743
:10656000C91A0B469B000B445B00D11ACBB23033E7
:10657000DBB203703B68134A82FB03129210DB17F5
:10658000D31A3B6012E0FB68002B0AD17B69012B18
:1065900007D13B697A6813442D221A700123FB60EE
:1065A00004E03B697A68134420221A703B69013B7E
:1065B0003B613B69002BC7DA00BF1C37BD465DF865
:1065C000047B70476766666680B400AF00BFBD4657
:1065D0005DF8047B7047000080B588B004AFF860B8
:1065E0007A601A460B46FB7213463B81FB680D4AE4
:1065F000934211D1FB7A63F07F03FB72FB7A9AB26C
:106600004FF47A7302933B8901937B6800930123D3
:106610003121F868FBF74EFF002318461037BD46BE
:1066200080BD00BF1401002080B58AB004AFF860BF
:106630007A601A460B46FB7213463B81FB680E4A92
:10664000934213D1FB7A63F07F03FB72FB7A9AB219
:106650004FF47A7302933B8901937B680093012383
:106660003121F868FCF74CF803467B617B691846DA
:106670001837BD4680BD00BF1401002080B584B02E
:1066800000AF78600523BB7300237B73786801F04B
:10669000B3F90346FB7397F90F30002B33D128E091
:1066A00007F10D017B680122D02000F032F803468B
:1066B000FB7397F90F30002B14D17B7B602B11D12A
:1066C0007A7B7B681A70786800F078F90346FB7370
:1066D00097F90F30002B10D1786801F005F80346C8
:1066E000FB730AE07B68DB6801209847BB7B013BBA
:1066F000BB73BB7B002BD3D100E000BFBB7B002B67
:1067000001D1FE23FB7397F90F3018461037BD46B1
:1067100080BD90B587B000AFB9607B600346FB7366
:106720001346BB81786801F067F90346FB7597F95A
:106730001730002B17D17B689B78012B03D0FB7B94
:1067400063F07F03FB737B685C687B685878BB8968
:10675000F97BBA68A0470346FB7597F91730002B01
:1067600001D0FC23FB7597F9173018461C37BD463E
:1067700090BD90B58DB000AFF860B9603B60134636
:10678000FB71FB790A2B01D90A23FB71386801F0F0
:1067900033F9034687F82F3097F92F30002B56D165
:1067A000FB68002B53D0BB68002B50D0FB79002B2B
:1067B00049D0BB681B783B753B689B78012B1AD08E
:1067C000002387F82B3011E097F82B30FA68134438
:1067D00097F82B20F9680A44127802F07F02D2B2AF
:1067E0001A7097F82B30013387F82B3097F82B204D
:1067F000FB799A42E8D3FB79012B0DD9FB7907F19C
:106800001401BA68F86800F0B3FFFB799BB25B0033
:106810009BB2013BBB8501E0FB79BB853B689C6873
:106820003B685878FB681978BB8D07F11402A047C4
:10683000034687F82F3097F92F30002B0BD0FC231D
:1068400087F82F3007E0FD2387F82F3003E0FF2380
:1068500087F82F3000E000BF97F92F301846343703
:10686000BD4690BD80B584B000AF03463960FB7172
:10687000386801F0C1F80346FB7397F90F30002B1D
:106880003FD107F10E033968184600F074F803464B
:10689000FB7397F90F30002B07D1BB7B002B04D083
:1068A000386800F056FB0346FB7397F90F30002B56
:1068B00027D1FB791946072001F082F80346002B07
:1068C00009D03B6803F13801FB793A68184600F0BB
:1068D00092F90346FB7397F90F30002B11D1FB7926
:1068E0001946182001F06CF80346002B09D03B68CC
:1068F00003F13801FB793A68184600F019FA0346AB
:10690000FB7397F90F3018461037BD4680BD80B530
:1069100084B000AF03463960FB71386801F06CF851
:106920000346FB7397F90F30002B1ED107F10E03BE
:106930003968184600F01FF80346FB7397F90F30CB
:10694000002B07D1BB7B002B04D0386800F001FB83
:106950000346FB7397F90F30002B06D1FB7939689A
:10696000184600F0C3FA0346FB7397F90F30184638
:106970001037BD4680BD80B584B000AF7860396007
:10698000386801F039F80346FB7397F90F30002B94
:106990000ED13B6801227968F420FFF7BAFE034666
:1069A000FB737B681B7803F00303DAB27B681A7011
:1069B00097F90F3018461037BD4680BD80B584B0BA
:1069C00000AF7860E023BB73B6237B73786801F077
:1069D00013F80346FB7397F90F30002B0DD107F125
:1069E0000D0107F10E007B680122FFF7C2FE03468E
:1069F000FB737B68DB680220984797F90F301846D5
:106A00001037BD4680BD80B58AB000AF0346B9607F
:106A10007A60FB7307F11C0300221A605A6007F1C9
:106A2000100300221A605A609A60786800F0E4FF50
:106A3000034687F8273097F92730002B24D1BB680D
:106A4000002B21D007F11C017B680822F720FFF7FB
:106A500060FE034687F8273097F92730002B16D1C0
:106A600007F1100207F11C031146184600F015F853
:106A70007B68103307F11001F87BBA6800F072F8F8
:106A8000034687F8273002E0FF2387F8273097F97D
:106A9000273018462837BD4680BD80B487B000AF88
:106AA000786039607B681B787B617B6801331B7879
:106AB0007B617B6802331B787B617B6803331B78C7
:106AC0007B617B6804331B787B617B6805331B78B3
:106AD0007B617B6806331B787B617B6807331B789F
:106AE0007B617B681B781B033B617B6801331B78F0
:106AF0001B01FB607B6802331B781B09DBB2BB60A8
:106B00003A69FB681A43BB681A433B681A607B68A2
:106B100003331B781B033B617B6804331B781B0129
:106B2000FB607B6805331B781B09DBB2BB603A69ED
:106B3000FB681A43BB681A433B685A607B6806339C
:106B40001B781B02FB607B6807331B783B613A694B
:106B5000FB681A433B689A6000BF1C37BD465DF86E
:106B6000047B704780B586B000AFB9607A603B6047
:106B70000346FB730023FB75BB68002B33D07B6897
:106B8000002B30D03B68002B2DD07B6800225A6050
:106B90007B6800221A607B6800229A60FB7B03F00E
:106BA0000703002B06D03968B86800F01FFA0246C8
:106BB0007B685A60FB7B03F00103002B06D0396829
:106BC000B86800F075FA02467B681A60FB7B03F038
:106BD0000403002B09D03968B86800F0D9FC0246DC
:106BE0007B689A6001E0FF23FB7597F91730184620
:106BF0001837BD4680BD80B586B000AF0346B9608A
:106C00007A60FB730123FB75FB7B03F00403002B0D
:106C100005D07968B86800F015F80346FB75FB7B72
:106C200003F00303002B07D0FB7B7A68B968184692
:106C300000F042F80346FB7597F9173018461837ED
:106C4000BD4680BD80B584B000AF78603960F22366
:106C50003B737B689B7803F00703DBB2BB7307F1E0
:106C60000E0107F10C003B680122FFF782FD03468D
:106C7000FB7397F90F30002B18D1F4233B73387B4B
:106C800007F10D013B680122FFF743FD0346FB734B
:106C900097F90F30002B09D107F10D0107F10C0016
:106CA0003B680122FFF765FD0346FB7397F90F3040
:106CB00018461037BD4680BD80B586B000AF03468C
:106CC000B9607A60FB73F423BB75B87D07F11501D9
:106CD0007B680122FFF71DFD0346FB7597F917300E
:106CE000002B1FD1FB7B03F00103002B05D007F124
:106CF0001503B968184600F08EF8FB7B03F0020319
:106D0000002B05D007F11503B968184600F0A0F86C
:106D100007F1150107F116007B680122FFF729FD35
:106D20000346FB7597F9173018461837BD4680BDE6
:106D300080B586B000AF0346B9607A60FB73F52377
:106D4000BB75B87D07F115017B680122FFF7E1FCF7
:106D50000346FB7597F91730002B1FD1FB7B03F01F
:106D60000803002B05D007F11503B968184600F099
:106D70001BF8FB7B03F01003002B05D007F1150374
:106D8000B968184600F02DF807F1150107F1160053
:106D90007B680122FFF7EDFC0346FB7597F917307E
:106DA00018461837BD4680BD80B483B000AF786008
:106DB00039607B681B785BB223F01C035AB23B68D6
:106DC000DB789B005BB203F01C035BB213435BB246
:106DD000DAB27B681A7000BF0C37BD465DF8047BE1
:106DE000704780B483B000AF786039607B681B78EF
:106DF0005BB203F01F035AB23B681B795B015BB2C5
:106E000013435BB2DAB27B681A7000BF0C37BD4621
:106E10005DF8047B704780B483B000AF7860396060
:106E20007B681B785BB223F01C035AB23B681B786B
:106E30009B005BB203F01C035BB213435BB2DAB29C
:106E40007B681A7000BF0C37BD465DF8047B704745
:106E500080B483B000AF786039607B681B785BB228
:106E600003F01F035AB23B685B785B015BB21343CC
:106E70005BB2DAB27B681A7000BF0C37BD465DF8B2
:106E8000047B704780B483B000AF786039607B6862
:106E90001B7803F00703DAB23B689A707B68023311
:106EA0001B789B10DBB203F00703DAB23B681A7061
:106EB0007B6802331B785B09DAB23B685A707B68E7
:106EC00003331B789B10DBB203F00703DAB23B6895
:106ED000DA707B6803331B785B09DAB23B681A719E
:106EE00000BF0C37BD465DF8047B704780B584B0A9
:106EF00000AF03463960FB71F423BB73B87B07F125
:106F00000D013B680122FFF704FC0346FB7397F970
:106F10000F30002B17D17B7B5BB223F003035AB2F7
:106F200097F9073003F003035BB213435BB2DBB2A4
:106F30007B7307F10D0107F10E003B680122FFF79B
:106F400018FC0346FB7397F90F3018461037BD46FF
:106F500080BD80B586B000AF786007F110017B6816
:106F60000422F220FFF7D5FB0346FB7597F9173093
:106F7000002B18D107F1080207F11003114618463B
:106F8000FFF780FF7868FFF719FD0346FB7597F957
:106F90001730002B07D107F108037968184600F075
:106FA00008F80346FB7597F9173018461837BD46A1
:106FB00080BD80B584B000AF786039603A68796888
:106FC0001F20FFF718FE0346FB7397F90F30002BC5
:106FD00006D13A6879681F20FFF7AAFE0346FB73C3
:106FE00097F90F3018461037BD4680BD80B489B080
:106FF00000AF786039602D4BBB6142F234137B6186
:107000007B685B68DB083A68128852009B1A3B6118
:107010003B68B3F902301A463B6903FB02F3002BCD
:1070200001DA03F2FF73DB123B617B685B681B09CB
:107030003A6812889B1AFB60FB68FA6802FB03F34C
:10704000002B01DA03F6FF731B131A463B68B3F9F2
:10705000043003FB02F3002B02DA03F57F533F33C6
:107060009B13FB603A69FB681A443B685A623B68B1
:107070005A6A13469B0013448033002B00DAFF3317
:107080001B12FB61FA69BB699A4202DABB69FB61B8
:1070900005E0FA697B699A4201DD7B69FB61FB6966
:1070A00018462437BD465DF8047B704760F0FFFF4B
:1070B0002DE9F04FADB000AFF867B967BF4BC7F827
:1070C000A830BF4BC7F8A430BB6F5B6A4FEAE374CC
:1070D000B3F5FA3344F1FF34C7E92634D7F89C20DE
:1070E000D7F8983003FB02F1D7F89C20D7F89830F6
:1070F00003FB02F3CC18D7F89820D7F89830A2FBFE
:10710000030163181946BB6FB3F910301BB24FEA85
:10711000E37403FB01F500FB04F22A44A0FB0334F3
:1071200022441446C7E92434C7E92434BB6FB3F9B9
:107130000E301BB24FEAE374D7F8982004FB02F13B
:10714000D7F89C2003FB02F21144D7F89820A2FB49
:1071500003340A1914464FEA444949EAD3394FEA3D
:107160004348D7E9243413EB080344EB0904C7E987
:107170002434BB6FB3F90C301BB24FEAE374DB006D
:10718000FB600023BB60D7E92434D7E90212C91899
:1071900042EB04020B461446C7E92434D7F89C207E
:1071A000D7F8983003FB02F1D7F89C20D7F8983035
:1071B00003FB02F3CC18D7F89820D7F89830A2FB3D
:1071C000030163181946BB6FB3F90A301BB24FEACB
:1071D000E37403FB01F500FB04F22A44A0FB033433
:1071E00022441446002B74F1000202DAFF3344F10A
:1071F00000044FEA132A4AEA046A4FEA242B554650
:107200005E46BB6FB3F908301BB24FEAE374D7F8A0
:10721000982004FB02F1D7F89C2003FB02F21144F2
:10722000D7F89820A2FB03340A19144622037A6780
:107230007A6F42EA13527A671B033B67D7E91C3423
:107240005B1944EB0604C7E926344FF000034FF402
:107250000044C7E92234D7E92212D7E92634C918F5
:1072600042EB0402BB6FDB889BB24FF0000403FBD0
:1072700002F501FB04F02844A1FB03340219144673
:10728000002B74F1000203DA13F1FF3344F101041F
:1072900062103A60E3177B6097E81800C7E926346C
:1072A000D7E92634234300F06581FB6F1B68C3F5E3
:1072B00080134FF00004C7E92034D7E92034E207F7
:1072C000FA66FA6E42EA5302FA66DB07BB66D7E952
:1072D0002434D7E91A12C91A62EB04020B46144689
:1072E000DB1844EB04045B1844EB0204A001F865CE
:1072F000F86D40EA9360F8659801B865D7E91656CD
:10730000ED1846EB04062B463446A0007865786DF0
:1073100040EA937078659B003B65D7E914345B18AD
:1073200044EB0204A000F864F86C40EA9370F8643F
:107330009B00BB64D7E912345D1844EB0206284673
:107340003146D7E92623F9F773FC03460C46C7E913
:107350002034BB6FB3F916301DB24FEAE576D7E99A
:107360002034002B74F1000206DA41F6FF714FF071
:1073700000025B1844EB02045A0B3A643A6C42EA8E
:10738000C4423A6463137B64D7E9103403FB06F10B
:1073900005FB04F20A44A5FB035693191E46D7E9E0
:1073A0002034002B74F100020CDA41F6FF714FF02B
:1073B00000025B1844EB020404E000BFC0C62D00CD
:1073C000C0D8A7005A0BBA63BA6B42EAC442BA6388
:1073D0006313FB63D7E90E3403FB06F105FB04F2EC
:1073E0000A44A5FB033422441446002B74F1000226
:1073F00006DA6FF07E414FF000025B1844EB0204A6
:107400005A0E3A633A6B42EAC4123A6363167B63DC
:10741000D7E90C34C7E92634BB6FB3F914301BB27B
:107420004FEAE374D7F8802004FB02F1D7F88420F8
:1074300003FB02F20A44D7F88010A1FB0334224474
:107440001446002B74F1000205DA50494FF0000297
:107450005B1844EB0204DA0CBA62BA6A42EA4432BC
:10746000BA62E314FB62D7E90A34C7E92434D7E9E6
:107470002012D7E92634C91842EB0402D7E9243494
:107480005B1844EB0204002B74F1000202DAFF33B4
:1074900044F100041A0A3A623A6A42EA04623A6221
:1074A00023127B62D7E90812BB6FB3F912301BB20B
:1074B0004FEAE37420017866786E40EA13707866CC
:1074C0001B013B66D7E918345B1844EB0204C7E99B
:1074D0002034D7E92034E20F11464FF000025B1848
:1074E00044EB020464104FEA3303194622460B466C
:1074F0001446DB1844EB04045B1844EB02046001FF
:10750000F861F86940EAD360F8615801B861D7E9D9
:107510000656ED1846EB04062B4634465B1844EB42
:107520000204002B74F1000202DA7F3344F10004FC
:10753000DA093A613A6942EA44623A61E3117B61ED
:10754000D7E90434C7F8AC30D7F8AC20D7F8A83066
:107550009A4204D2D7F8A830C7F8AC300EE0D7F87A
:10756000AC20D7F8A4309A4208D9D7F8A430C7F88D
:10757000AC3003E0D7F8A830C7F8AC30D7F8AC305F
:107580001846B437BD46BDE8F08F00BFFFFF0700C7
:1075900080B48BB000AF786039604FF4C8333B6281
:1075A0003B685B6AA3F59633FB617B689B689B0332
:1075B000BB613B68B3F91E301B057B613B68B3F9C7
:1075C00020301A46FB6903FB02F33B61BA697B6911
:1075D000D21A3B69D31A03F58043002B02DA03F574
:1075E000FF437F33DB13FB603B6893F922301A467D
:1075F000FB6903FB02F3002B01DA03F2FF339B125A
:10760000BB613B681B7F1A46FB6903FB02F3002B3F
:1076100001DA03F2FF73DB127B617B6903F5004340
:10762000BA6902FB03F3002B01DA03F2FF339B126A
:1076300003F500133B613B68B3F91A301A463B6906
:1076400003FB02F303F50053002B02DA03F57F532B
:107650003F339B13BB61FB68BA6902FB03F37B6199
:107660007B69002B02DA03F5FF437F33DB131A46F5
:107670007B69002B02DA03F5FF437F33DB1303FB47
:1076800002F3002B00DA7F33DB113B613B681B7E8A
:107690001A463B6903FB02F3002B00DA0F331B1180
:1076A0005B421A467B691344FB60FB6823EAE37381
:1076B000FB60FB68B3F1C85FA8BF4FF0C853FB6025
:1076C000FB68002B01DA03F6FF731B137B627A6AF7
:1076D0003B6A9A4201D93B6A7B627B6A18462C3727
:1076E000BD465DF8047B704780B58AB000AF786016
:1076F000882387F8263007F10C0300221A605A60AD
:107700009A60DA601A615A611A8307F10C0197F8DE
:1077100026007B681A22FEF7FCFF034687F8273015
:1077200097F92730002B1DD107F10C037968184613
:1077300000F049F8E12387F8263007F10C0197F8AB
:1077400026007B680722FEF7E4FF034687F8273010
:1077500097F92730002B05D107F10C0379681846FB
:1077600000F0E0F897F9273018462837BD4680BD6D
:1077700080B487B000AFF860B9607A60FB70012315
:10778000FB7516E0FB7D5B00013BBA681344FA7D94
:10779000F9680A4412781A70FB7D5B001A46BB68D0
:1077A0001344FA7D79680A4412781A70FB7D01331C
:1077B000FB75FA7DFB789A42E4D300BF1C37BD46C7
:1077C0005DF8047B704780B485B000AF78603960A5
:1077D0003B681033FB607B6801331B781B021AB2D5
:1077E0007B681B781BB213431BB29AB2FB681A80EA
:1077F0007B6803331B781B021AB27B6802331B7849
:107800001BB213431AB2FB685A807B6805331B789E
:107810001B021AB27B6804331B781BB213431AB2E3
:10782000FB689A807B6807331B781B021AB27B685F
:1078300006331B781BB213431BB29AB2FB68DA8083
:107840007B6809331B781B021AB27B6808331B78EC
:107850001BB213431AB2FB681A817B680B331B7887
:107860001B021AB27B680A331B781BB213431AB28D
:10787000FB685A817B680D331B781B021AB27B6848
:107880000C331B781BB213431AB2FB689A817B68D6
:107890000F331B781B021AB27B680E331B781BB2A6
:1078A00013431AB2FB68DA817B6811331B781B0221
:1078B0001AB27B6810331B781BB213431AB2FB68F1
:1078C0001A827B6813331B781B021AB27B6812334F
:1078D0001B781BB213431AB2FB685A827B681533BC
:1078E0001B781B021AB27B6814331B781BB213433C
:1078F0001AB2FB689A827B6817331B781B021AB294
:107900007B6816331B781BB213431AB2FB68DA820A
:107910007B685A7EFB681A7600BF1437BD465DF857
:10792000047B704780B487B000AF786039603B68F3
:1079300010337B617B6801331B781B021AB27B68B2
:107940001B781BB213431AB27B695A837B689A78FF
:107950007B691A777B6803331B785BB29BB21B0190
:107960009BB27B827B6804331B781BB203F00F034E
:107970003B827A8A3B8A13431AB27B69DA837B683B
:1079800005331B785BB29BB21B019BB2FB817B680A
:1079900004331B781B09DBB2BB81FA89BB89134313
:1079A0001AB27B691A847B6806331B785AB27B69EA
:1079B00083F8222000BF1C37BD465DF8047B70476A
:1079C00080B485B000AF03460A46FB711346BB7115
:1079D0000023FB73FA79BB791340DBB2002B02D092
:1079E0000123FB7301E00023FB73FB7B1846143774
:1079F000BD465DF8047B704780B485B000AF786009
:107A00007B68002B0BD07B685B68002B07D07B6802
:107A10009B68002B03D07B68DB68002B02D1FF231F
:107A2000FB7301E00023FB7397F90F3018461437FE
:107A3000BD465DF8047B704790B587B000AFF86035
:107A40007A601A460B46FB7213463B81FB685C6802
:107A5000FB6898683B89F97A7A68A04778617B6906
:107A600018461C37BD4690BD90B587B000AFF86092
:107A70007A601A460B46FB7213463B81FB681C6812
:107A8000FB6898683B89F97A7A68A04778617B69D6
:107A900018461C37BD4690BD80B483B000AF034686
:107AA000FB80B7F9063007EE903AF8EEE77AB3EECE
:107AB000007AC7EE876AF0EE667AB0EE670A0C3796
:107AC000BD465DF8047B704780B584B000AF786038
:107AD0000B46FB7007F1080201231F217868FFF7AE
:107AE000ABFFF860FB68002B0FD1FB7803F00303BA
:107AF000DAB23B7A62F387133B7207F10802012383
:107B00001F217868FFF7B0FFF860FB681846103750
:107B1000BD4680BD80B586B000AF78600B46FB7077
:107B200007F11002012320217868FFF785FF7861B3
:107B30007B69002B07D107F10C0201232321786810
:107B4000FFF77AFF78617B69002B28D1FB78002B47
:107B500007D13B7C6FF3C3033B743B7B43F00803CB
:107B60003B73FB78012B07D13B7C6FF3C3033B7462
:107B70003B7B6FF3C3033B73FB78022B07D13B7C4A
:107B800043F008033B743B7B6FF3C3033B7307F184
:107B90001002012320217868FFF766FF78617B6976
:107BA000002B07D107F10C02012323217868FFF78E
:107BB0005BFF78617B6918461837BD4680BD80B58C
:107BC00084B000AF78600B46FB7007F10802012318
:107BD00020217868FFF730FFF860FB68002B0FD199
:107BE000FB7803F00F03DAB23B7A62F307133B72C0
:107BF00007F10802012320217868FFF735FFF860BC
:107C0000FB6818461037BD4680BD80B584B000AF14
:107C100078600B46FB7007F1080201232321786886
:107C2000FFF70AFFF860FB68002B0FD1FB7803F029
:107C30000303DAB23B7A62F305133B7207F10802E1
:107C4000012323217868FFF70FFFF860FB681846CF
:107C50001037BD4680BD80B584B000AF78600B465C
:107C6000FB7007F10802012323217868FFF7E4FE87
:107C7000F860FB68002B0FD1FB7803F00103DAB248
:107C80003B7A62F3C7133B7207F1080201232321F9
:107C90007868FFF7E9FEF860FB6818461037BD46C4
:107CA00080BD80B584B000AF7860396007F108020C
:107CB000012327217868FFF7BFFEF8603B7AC3F302
:107CC000C003DBB21A463B681A70FB6818461037CF
:107CD000BD4680BD80B584B000AF786039600623B2
:107CE0003A6828217868FFF7A7FEF860FB68184615
:107CF0001037BD4680BD80B584B000AF7860396074
:107D000001233A680F217868FFF796FEF860FB6858
:107D100018461037BD4680BD90B5EFB00CAFF9F7EF
:107D200047F9CF4A07F5827307CA03C31A700023C5
:107D3000C7F81C310023C7F884310023C7F880310D
:107D40000D23C7F87C310023C7F878310023C7F82A
:107D500074310023C7F87031C24A07F1FC0392E87E
:107D6000030018600433197007F1A0035B2200219F
:107D7000184601F075F9BC4A07F1980392E8030030
:107D800083E803000023C7F86C312D2387F8943073
:107D90002B2387F8903007F18803B44A92E8030058
:107DA00083E803004FF00003C7F8683107F15C0374
:107DB000AF4A07CA03C31A804FF00003C7F8643103
:107DC00007F15003AB4A07CA03C31A800233120CEF
:107DD0001A7007F14C03A84A126811461980023341
:107DE000120C1A7007F14803A34A12681146198051
:107DF0000233120C1A7007F144039F4A12681146AD
:107E000019800233120C1A7007F140039B4A1A6062
:107E100007F13C03994A1A6007F13803974A1A6040
:107E200007F13403944A1268114619800233120C88
:107E30001A7007F13003924A126811461980023312
:107E4000120C1A7007F124038E4A07CA03C31A8062
:107E500007F11C038C4A92E8030018600433198070
:107E600002330A0C1A700023C7F860310023C7F8E8
:107E70005C314FF00003C7F818314FF00003C7F82A
:107E800014314FF00003C7F858314FF00003C7F822
:107E900054310023C7F850310023C7F84C314FF05C
:107EA0000003C7F848314FF00003C7F844310023FE
:107EB000C7F840310023C7F83C310023C7F83831F8
:107EC0000023C7F834310023C7F830310023C7F846
:107ED0002C3100F099FC00F0D3FD00F0A1FD00F082
:107EE000F1FC00F05DFD012268496948FCF722FBC6
:107EF0006848F9F775FA0023C7F828313B1D1A4680
:107F00000023136053609360D36013615361FDF7E6
:107F1000B3FDFEF74DF8FEF7E7F95F4B1B680A2B40
:107F200040F3EC804FF00003C7F810315948F9F7DF
:107F30000DFB07EE900AF8EE677AC7ED447AD7F8A2
:107F40002831002B27D1D7F81001F8F7F5FA3CA318
:107F5000D3E90023F8F744FB03460C4618462146B4
:107F600039A3D3E90023F8F789F903460C461846EC
:107F70002146F8F70DFE0346C7F8183197ED567AFB
:107F8000D7ED467A77EE277AC7ED567AD7F8503193
:107F90000133C7F85031D7F82831012B27D1D7F852
:107FA0001001F8F7C9FA2AA3D3E90023F8F718FB60
:107FB00003460C461846214627A3D3E90023F8F7C9
:107FC0005DF903460C4618462146F8F7E1FD0346E5
:107FD000C7F8143197ED557AD7ED457A77EE277AC1
:107FE000C7ED557AD7F84C310133C7F84C312B4BDC
:107FF0001B68C82B0CDDFEF79BF8D7F83431013332
:10800000C7F83431254B00221A600023C7F82C3101
:10801000224B1B68642B08DDD7F82C31002B04D1D0
:10802000FEF79EF90123C7F82C31D7F82831002B31
:1080300036D13B1D01221A6035E000BFAFF300804E
:10804000EE3B2B0E0CC5A23F65C746205ED7F23F24
:10805000294E20B26921683FA4C16D6DE179C33F0B
:108060002CAB000838AB000840AB000848AB000858
:1080700054AB000860AB00086CAB00082020203037
:1080800070AB000874AB000880AB0008C002002091
:10809000DC01002088010020BC000020C00000207E
:1080A0003B1D02221A603B1D01225A603B1D00222B
:1080B000DA603B1D07229A603B1D00221A613B1DBE
:1080C00000225A613B1D1946C248F9F74DFA034692
:1080D000002B01D000F064FDBE48F9F781F9BE4BDA
:1080E00000221A60D7F828310133C7F82831D7F8B1
:1080F0002831012B02DD0023C7F82831F8F7B2FF41
:108100000246D7F87831D31A40F2E232934240F275
:108110009780D7F83031002B40F09280D7F850315B
:10812000002B0BDDD7F8503107EE903AB8EEE77A26
:10813000D7ED566AC6EE877AC7ED517AD7F84C313B
:10814000002B53DDD7F84C3107EE903AB8EEE77AC2
:10815000D7ED556AC6EE877AC7ED527A9F4B1A68FB
:10816000D7F8343192FBF3F31846F8F7D3F9034606
:108170000C4644EC103B01F01FFC54EC103B18463D
:108180002146F8F7DDFC0346C7F84031944B1A68E6
:10819000D7F8343192FBF3F31846F8F7BBF90346EE
:1081A0000C4644EC103B01F007FC54EC103B184625
:1081B0002146F8F7C5FC0346C7F83C31894B1A68DD
:1081C000D7F8343192FBF3F31846F8F7A3F90346D6
:1081D0000C4644EC103B01F0EFFB54EC103B18460E
:1081E0002146F8F7ADFC0346C7F8383107F13403F0
:1081F00097ED510A1846FDF763FB07F1300397ED41
:10820000520A1846FDF7DAFB07F1480207F14C0164
:1082100007F14400D7F838310193D7F84031009383
:10822000D7F83C31FDF7C4FF07F1380207F13C01F4
:1082300007F140031846FEF7D5F80123C7F830319F
:10824000F8F710FF0246D7F87831D31AB3F57A7FE2
:108250006DD3D7F870310133C7F8703107F1FC03E3
:10826000D7F870216049184600F002FF07F1880432
:1082700007F1FC0207F5827107F1A00007F1300356
:108280000A9307F13403099307F11C03089307F1DC
:108290005003079307F15C03069307F13803059336
:1082A00007F13C03049307F14003039307F14403F0
:1082B000029307F14803019307F14C03009323460F
:1082C000FDF77EF907F1A0014FF47A735B2247486E
:1082D000FCF7A3F8F8F7C6FE0346C7F87831002389
:1082E000C7F850310023C7F84C310023C7F83431A8
:1082F0004FF00003C7F858314FF00003C7F854316E
:10830000374B00221A60354B00221A60354B002291
:108310001A600023C7F83031354BD3ED007AD7F817
:108320004011D7F85C01B0EE670AFDF779FC314BDC
:108330001B68033B304AD35CDBB22A2B40F0378208
:108340002D4B5B78DBB2C7F884312A4B1B68023BAC
:10835000294AD35CDBB21846FDF708F803461C0136
:10836000244B1B68013B244AD35CDBB21846FCF764
:10837000FDFF03462344C7F81C310223C7F824310C
:1083800010E01D4AD7F8243113441B78DBB21A469B
:10839000D7F884315340C7F88431D7F824310133FA
:1083A000C7F82431134B1B68DA1ED7F824319A42E0
:1083B000E7DCD7F81C21D7F884319A4240F0DF81FE
:1083C0000123C7F86C310023C7F880310023C7F8B8
:1083D000803129E088010020BC000020B800002086
:1083E000B0000020B400002028AB0008DC01002011
:1083F000AC000020BC0200204C020020A74AD7F8A5
:10840000803113441B78DAB207F19801D7F8803134
:108410000B441B789A4202D00023C7F86C31D7F87E
:1084200080310133C7F88031D7F88031062BE5DD84
:10843000D7F86C31012B40F0A281984BDB79DBB28D
:108440002C2B23D0954BDB79DAB207F188031A7015
:10845000924B1B7ADAB207F188035A708F4B5B7A22
:10846000DAB207F18803DA708C4B9B7ADAB207F143
:1084700088031A71894BDB7ADAB207F188039A71A3
:10848000864B1B7BDAB207F18803DA710D23C7F83C
:108490007C3104E0D7F87C310133C7F87C317F4A66
:1084A000D7F87C3113441B78DBB22C2BF2D1D7F8F0
:1084B0007C310133C7F87C310023C7F8803116E0E6
:1084C000764AD7F87C3113441B78D9B207F1780289
:1084D000D7F8803113440A461A70D7F87C3101333B
:1084E000C7F87C31D7F880310133C7F880316B4A47
:1084F000D7F87C3113441B78DBB22C2BE0D1D7F8B2
:108500008031002B08D007F17803D7F88011184686
:10851000FCF78EFD87ED5A0AD7F87C310133C7F896
:108520007C315E4AD7F87C3113441B78DBB24E2B8A
:1085300002D12B2387F89030584AD7F87C31134466
:108540001B78DBB2532B02D12D2387F8903097F89C
:10855000902007F15C0397ED5A0A0A211846FCF7B0
:108560004FFE4E4AD7F87C3113441B78DBB22C2BDC
:1085700004D0D7F87C310133C7F87C31D7F87C318F
:108580000133C7F87C310023C7F8803116E0434A35
:10859000D7F87C3113441B78D9B207F16802D7F8B9
:1085A000803113440A461A70D7F87C310133C7F87A
:1085B0007C31D7F880310133C7F88031374AD7F89A
:1085C0007C3113441B78DBB22C2BE0D1D7F88031FF
:1085D000002B08D007F16803D7F880111846FCF784
:1085E00027FD87ED590AD7F87C310133C7F87C3174
:1085F0002A4AD7F87C3113441B78DBB2452B02D1D1
:108600002B2387F89430254AD7F87C3113441B7804
:10861000DBB2572B02D12D2387F8943097F89420A2
:1086200007F1500397ED590A0B211846FCF7E8FDB6
:108630001A4AD7F87C3113441B78DBB22C2B04D0B8
:10864000D7F87C310133C7F87C31D7F87C3101335E
:10865000C7F87C310023C7F8803116E0D7F87C31A9
:108660000133C7F87C310D4AD7F87C3113441B78AD
:10867000DBB22C2BF2D1D7F87C310133C7F87C3137
:10868000D7F880310133C7F88031D7F88031022B19
:10869000E9DD0023C7F8803119E000BF4C0200205B
:1086A000534AD7F87C3113441B78D9B207F124021E
:1086B000D7F8803113440A461A70D7F87C31013359
:1086C000C7F87C31D7F880310133C7F88031484A88
:1086D000D7F87C3113441B78DBB22C2BE0D1D7F8D0
:1086E0008031002B08D007F11C0207F12403D7F8D2
:1086F00080111846FCF75CFE3E4B1B681846F7F7E6
:108700001BFF37A3D3E90023F8F7DCF90346002B5E
:108710000CD1384B1B681846F7F70EFF32A3D3E98C
:108720000023F8F7EDF90346002B0FD0324BD3EDC1
:10873000007A9FED327AF4EEC77AF1EE10FA05DD99
:10874000D7F860310133C7F8603102E00023C7F881
:108750006031D7F86031042B11DDD7F85C31002B84
:108760000DD101224FF480612548F9F7FDFDF8F79E
:1087700079FC0346C7F874310123C7F85C31002344
:10878000C7F820310AE01A4AD7F8203113440022F2
:108790001A70D7F820310133C7F82031194B1B6804
:1087A000D7F820219A42EEDB164B00221A60F8F728
:1087B00059FC0246D7F87431D31A42F20F72934231
:1087C0007FF6ABABD7F85C31012B7FF4A6AB002270
:1087D0004FF480610A48F9F7C7FDFFF79EBB00BF61
:1087E000B4AD669DF1F93140ACADD85F76EF324063
:1087F0004C020020A8000020AC00002000401C46D5
:1088000000040048BC02002080B596B000AF07F11C
:10881000300328220021184600F022FC07F11C0337
:1088200000221A605A609A60DA601A613B460022A0
:108830001A605A609A60DA601A615A619A6102237A
:108840003B6301233B6410237B640223FB6400230E
:108850003B654FF460137B6507F130031846FAF768
:1088600033FB0346002B01D000F09AF90F23FB6184
:1088700002233B6200237B624FF48063BB620023D0
:10888000FB6207F11C0302211846FBF70BFA0346B3
:10889000002B01D000F084F9A1233B600023BB60D2
:1088A0004FF480733B610023FB603B461846FBF7A7
:1088B0002FFC0346002B01D000F072F900BF58379F
:1088C000BD4680BD80B58AB000AF07F11C03002211
:1088D0001A605A609A603B1D00221A605A609A60C2
:1088E000DA601A615A612D4B4FF0A0421A602B4B8F
:1088F00000225A60294B00229A60284B00221A61FC
:10890000264B0022DA61254B00225A62234B0022BB
:108910001A63224B0122DA62204B0022DA601F4BDD
:1089200001221A621D4B00225A631C4B04225A6119
:108930001A4B00229A61194B00229A631748F8F7E4
:10894000BFFB0346002B01D000F02AF90023FB6196
:1089500007F11C0319461148F9F7C4F80346002B28
:1089600001D000F01DF901237B600123BB600023CF
:108970003B610023FB6000237B610023BB613B1D47
:1089800019460648F8F7F0FD0346002B01D000F029
:1089900007F900BF2837BD4680BD00BF8801002011
:1089A00080B500AF1B4B1C4A1A601A4B1B4A5A6019
:1089B000184B00229A60174B0122DA60154B0022F7
:1089C0001A61144B00225A61124B00229A61114B1A
:1089D0000022DA610F4B00221A620E48F9F7DCFC24
:1089E0000346002B01D000F0DBF800210948FAF71C
:1089F000D1F90346002B01D000F0D2F80021054840
:108A0000FAF713FA0346002B01D000F0C9F800BFB3
:108A100080BD00BF14010020005400400E0900205A
:108A200080B500AF144B154A1A60134B4FF4E13276
:108A30005A60114B00229A600F4B0022DA600E4BF5
:108A400000221A610C4B0C225A610B4B00229A61D6
:108A5000094B0022DA61084B00221A62064B002201
:108A60005A620548FBF788FC0346002B01D000F052
:108A700097F800BF80BD00BFDC0100200038014036
:108A800080B58AB000AF07F1140300221A605A6063
:108A90009A60DA601A613E4A3D4B5B6943F40023F9
:108AA00053613B4B5B6903F400233B613B69384AEC
:108AB000374B5B6943F480035361354B5B6903F4C7
:108AC0008003FB60FB68324A314B5B6943F400333F
:108AD00053612F4B5B6903F40033BB60BB682C4AC6
:108AE0002B4B5B6943F480235361294B5B6903F48F
:108AF00080237B607B68002220214FF09040F9F7B3
:108B000033FC00224FF606412248F9F72DFC4FF4C2
:108B100000537B61204BBB610023FB6107F1140311
:108B200019461E48F9F7AAFA0C237B610223BB61A0
:108B30000023FB6103233B6207237B6207F11403DD
:108B400019464FF09040F9F799FA20237B610123F1
:108B5000BB610023FB6100233B6207F1140319464C
:108B60004FF09040F9F78AFA4FF606437B610123F4
:108B7000BB610023FB6100233B6207F1140319462C
:108B80000448F9F77BFA00BF2837BD4680BD00BF17
:108B900000100240000400480000211000080048B6
:108BA00080B400AF00BFBD465DF8047B7047000095
:108BB00080B582B000AF0F4A0E4B9B6943F00103B2
:108BC00093610C4B9B6903F001037B607B68094A4E
:108BD000084BDB6943F08053D361064BDB6903F03C
:108BE00080533B603B680720F9F7C8F900BF08379E
:108BF000BD4680BD0010024080B58AB000AF7860ED
:108C000007F1140300221A605A609A60DA601A6150
:108C10007B681B68B3F1A04F24D1144A134B5B69E6
:108C200043F080535361114B5B6903F080533B6108
:108C30003B690E4A0D4B5B6943F4003353610B4BA8
:108C40005B6903F40033FB60FB6803237B61032350
:108C5000BB610023FB6107F1140319464FF09040FC
:108C6000F9F70CFA00BF2837BD4680BD001002405E
:108C700080B58AB000AF786007F1140300221A6053
:108C80005A609A60DA601A617B681B68264A9342D0
:108C900045D1264A254B5B6943F400335361234B8E
:108CA0005B6903F400333B613B69204A1F4B5B69FE
:108CB00043F4802353611D4B5B6903F48023FB6005
:108CC000FB684FF400437B611223BB610123FB610E
:108CD00003233B6204237B6207F1140319464FF020
:108CE0009040F9F7CBF980237B611223BB6101230C
:108CF000FB6103233B6204237B6207F114031946E3
:108D00000B48F9F7BBF9094A084BDB6943F4001338
:108D1000D361064BDB6903F40013BB60BB6800BF83
:108D20002837BD4680BD00BF0054004000100240FF
:108D30000004004880B58AB000AF786007F11403E2
:108D400000221A605A609A60DA601A617B681B68B8
:108D50001B4A93422FD11B4A1A4B9B6943F4804311
:108D60009361184B9B6903F480433B613B69154A4F
:108D7000144B5B6943F400235361124B5B6903F4AA
:108D80000023FB60FB6830237B610223BB6100236F
:108D9000FB6103233B6207237B6207F1140319463F
:108DA0000948F9F76BF9002200212520F9F7F1F8BD
:108DB0002520F9F70AF900BF2837BD4680BD00BF5E
:108DC00000380140001002400008004880B400AFA5
:108DD00000BFBD465DF8047B704780B400AFFEE77E
:108DE00080B400AFFEE780B400AFFEE780B400AF10
:108DF000FEE780B400AF00BFBD465DF8047B70475E
:108E000080B400AF00BFBD465DF8047B704780B4FE
:108E100000AF00BFBD465DF8047B704780B500AF72
:108E2000F8F70CF9054B1B680133044A1360044B37
:108E30001B680133024A136000BF80BDBC000020E4
:108E4000C000002080B582B000AF1C48FBF7FAFBE1
:108E50001A4B1B689B8C9BB2FB70FB78242B12D1A6
:108E600000237B6007E0164A7B68134400221A70D7
:108E70007B6801337B60134B1B687A689A42F2DB94
:108E8000104B00221A600F4B1B680D49FA78CA5428
:108E90000C4B1B6801330B4A13600A4B1B686C2B8D
:108EA00002DD084B00221A60012207490348FBF744
:108EB00041FB00BF0837BD4680BD00BFDC0100207C
:108EC0004C020020BC020020C002002080B584B00B
:108ED00000AF7860114B1B68002B02D10F4B104A7A
:108EE0001A600E4B1B68FB600C4B1A687B681344BE
:108EF0006A46934207D900F089F802460C231360B2
:108F00004FF0FF3306E0054B1A687B681344034AB1
:108F10001360FB6818461037BD4680BDC4000020B2
:108F2000C802002080B400AF1F4A1F4BD3F888301E
:108F300043F47003C2F888301C4A1C4B1B6843F092
:108F4000010313601949194B5A68194B13404B60C0
:108F5000164A164B1B6823F0847323F48033136086
:108F6000124A124B1B6823F4802313600F4A0F4BE5
:108F70005B6823F4FE0353600C4A0C4BDB6A23F05E
:108F80000F03D3620949094B1A6B0A4B13400B6359
:108F9000064B00229A60044B4FF000629A6000BFBB
:108FA000BD465DF8047B704700ED00E00010024014
:108FB0000CC07FF8CCFC00FFDFF834D0002103E0C8
:108FC0000C4B5B58435004310B480C4B42189A42EF
:108FD000F6D30B4A02E0002342F8043B094B9A42C5
:108FE000F9D3FFF79FFF00F017F8FEF795FEFEE7B5
:108FF0000030002048AC0008000000207400002071
:1090000074000020C8020020FEE70000014B186831
:10901000704700BF0C00002070B50D4E0D4CA41B16
:10902000A4100025A54209D10B4E0C4C01F070FD97
:10903000A41BA4100025A54205D170BD56F825300B
:1090400098470135EEE756F8253098470135F2E7A5
:1090500040AC000840AC000840AC000844AC00083C
:1090600002440346934200D1704703F8011BF9E71D
:109070000EB400B59CB04FF402711DABADF81410E6
:10908000029006906FF000410A48049107914FF654
:10909000FF7153F8042BADF816100068019302A974
:1090A00000F066F8029B00221A701CB05DF804EB19
:1090B00003B070470C0000202DE9F0478E689E42F7
:1090C00082460C469146984635D88A8912F4906FAC
:1090D00031D0256809696F1A6569022305EB4505DA
:1090E00095FBF3F508F101033B449D4238BF1D4653
:1090F000530531D5294600F039FB064650B90C23FB
:10910000CAF80030A38943F04003A3814FF0FF3039
:10911000BDE8F0873A46216900F0B4FAA38923F448
:10912000906343F08003A381266165613E44ED1B9B
:109130002660A5604646464528BF46463246494613
:10914000206800F0AAFAA3689B1BA36023681E4452
:1091500026600020BDE8F0872A4600F065FB064641
:109160000028E1D12169504600F0B2FAC7E70000BB
:109170002DE9F04F9DB0804603938B891C060D4668
:1091800016460FD50B696BB9402100F0EFFA286045
:10919000286128B90C23C8F800304FF0FF30C5E033
:1091A00040236B610023099320238DF8293030235D
:1091B0008DF82A304FF0010B37463C4614F8013B3E
:1091C000002B3CD1B7EB060A0BD05346324629465A
:1091D0004046FFF771FF013000F0A380099B534424
:1091E00009933B78002B00F09C8000234FF0FF3266
:1091F00004930793059206938DF853301A93052232
:1092000021785048F6F7E4FF671C049BD8B9D906CB
:1092100044BF20228DF853201A0744BF2B228DF81B
:10922000532022782A2A16D0079A00210A2027469E
:1092300001343B78303B092B51D9C9B111E0252BC2
:10924000C0D02746B9E73F4A801A0BFA00F018430E
:1092500004903C46D3E7039A111D12680391002A3B
:1092600001DB079204E0524243F0020307920493A9
:109270003B782E2B0ED17B782A2B07F1010132D1BE
:10928000039B1A1D1B680392002BB8BF4FF0FF33DE
:10929000023705932C4C397803222046F6F798FFC5
:1092A00038B14023001B03FA00F0049B03430493EE
:1092B0000137397825488DF8281006227E1CF6F7EC
:1092C00087FF002835D0224BFBB9039B073323F0DF
:1092D000070308330393099B4B4409936CE700FB96
:1092E00002320121A3E70023059318460A240F4602
:1092F00001313A78303A092A03D9002BCAD00590B7
:10930000C8E704FB00200123F1E703AB00932A46E2
:10931000104B04A94046AFF30080B0F1FF3F8146F7
:10932000D9D1AB895B063FF538AF09981DB0BDE8D0
:10933000F08F03AB00932A46064B04A9404600F089
:1093400081F8EAE7C0AB0008C6AB0008CAAB00086A
:1093500000000000B99000082DE9F04791461F4633
:109360008A680B69DDF820809342B8BF1346C9F8BC
:10937000003091F8432006460C4612B10133C9F87B
:1093800000302368990642BFD9F800300233C9F88B
:109390000030256815F0060507D104F1190AE368C5
:1093A000D9F800209B1A9D4229DB94F843302268AB
:1093B000003318BF012392062ED404F1430239462C
:1093C0003046C047013021D02368E568D9F8002035
:1093D00003F00603042B08BFAD1AA36822690CBF73
:1093E00025EAE57500259342C4BF9B1AED184FF09E
:1093F00000091A344D451BD10020BDE8F087012338
:10940000524639463046C047013003D14FF0FF3055
:10941000BDE8F0870135C2E7E1185A1C302081F819
:109420004300224494F8451082F843100233C4E705
:109430000123224639463046C0470130E6D009F1C3
:109440000109D7E72DE9F04317460A7E85B06E2A59
:10945000984606460C460C9B01F1430E00F0BC807A
:109460001AD8632A2ED00AD8002A00F0C880582AB9
:1094700000F08A8004F1420584F842202AE0642A40
:1094800001D0692AF6D121681A6811F0800F23D023
:10949000111D1960136827E0732A00F0B48008D802
:1094A0006F2A2AD0702AE5D10A6842F020020A60A9
:1094B00003E0752A21D0782ADCD1782284F845206F
:1094C0006E4964E01A6801F14205111D19601368C4
:1094D00084F842300123A3E011F0400F02F10401AF
:1094E0001960D7D0B2F90030002B03DA2D225B428D
:1094F00084F8432062490A2217E02068196810F0B6
:10950000800F03D0081D18600B6806E010F0400FB4
:1095100001F104001860F7D00B8859496F2A14BF75
:109520000A220822002084F843006568A560002D07
:10953000C0F29C80206820F004002060002B3FD106
:10954000002D40F095807546082A0BD12368DA0774
:1095500008D5236962689A42DEBF302305F8013CD2
:1095600005F1FF35AEEB05032361CDF800803B46E6
:1095700003AA21463046FFF7EFFE013055D14FF0E8
:10958000FF3005B0BDE8F08381F845203C492268F2
:10959000186812F0800F00F104051D6001D0036807
:1095A00002E05506FBD50388D00744BF42F02002F5
:1095B00022601BB9226822F0200222601022B1E74B
:1095C0007546B3FBF2F002FB1033CB5C05F8013DAE
:1095D00003460028F5D1B7E708681A68496910F012
:1095E000800F04D0101D18601368196007E010F098
:1095F000400F02F1040018601368F6D019800023B0
:1096000023617546B1E71A68111D19601568626813
:1096100000212846F6F7DCFD08B1401B6060636856
:109620002361002384F843309FE723692A463946A3
:109630003046C0470130A2D023689B0707D50025DC
:1096400004F11909E368039A9B1A9D4205DBE0685F
:10965000039B9842B8BF184693E701234A46394610
:109660003046C04701308AD00135EBE7002BA7D147
:109670000B7884F8423004F1420565E7E2AB00085C
:10968000D1AB000810B5431E0A44914200D110BD71
:1096900011F8014B03F8014FF7E7884210B501EBD1
:1096A000020303D8421E99420CD110BD9842F9D250
:1096B0008118D21AD34200D110BD13F8014D01F820
:1096C000014DF7E711F8014B02F8014FEBE70000FD
:1096D00038B50546002945D051F8043C0C1F002B35
:1096E000B8BFE41800F0D6F81F4A1368104633B923
:1096F000636014602846BDE8384000F0CCB8A3424F
:109700000CD921686218934204BF1A685B686360D1
:1097100004BF521822600460ECE713465A680AB18D
:10972000A242FAD919685818A0420BD12068014406
:10973000581882421960DDD1106852685A6001449D
:109740001960D7E702D90C232B60D3E720682118D2
:109750008A4204BF11685268626004BF0918216020
:109760005C60C7E738BD00BFC800002070B5CD1CE5
:1097700025F0030508350C2D38BF0C25002D0646B5
:1097800001DBA94203D90C233360002070BD00F037
:1097900081F8234A1468214691B9224C23681BB9E9
:1097A000304600F067F820602946304600F062F845
:1097B000431C26D10C233360304600F06CF8E4E7FC
:1097C0000B685B1B1AD40B2B0FD90B60CD50CC1838
:1097D000304600F060F804F10B00231D20F0070074
:1097E000C31A1BD05A42E25070BD8C420DBF636851
:1097F0004B686360136018BF0C46E9E70C46496884
:10980000CAE7C41C24F00304A04205D0211A304644
:1098100000F030F80130CDD02560D9E770BD00BF31
:10982000C8000020CC000020F8B5074614460E46BC
:1098300021B91146BDE8F840FFF798BF22B9FFF7FC
:1098400047FF25462846F8BD00F026F884420FD988
:1098500021463846FFF78AFF05460028F2D03146F8
:109860002246FFF70FFF31463846FFF731FFE9E7A1
:109870003546E7E738B5064C002305460846236021
:10988000FFF724FB431C02D1236803B12B6038BDD2
:10989000C40200207047704751F8040C0028A0F162
:1098A0000400BCBF0B58C018704700000000000047
:1098B00051EC100B2DE9F041C1F30A57A7F2FF3626
:1098C000132E10EE108A0C4610EE105A35DC002EC6
:1098D00017DA35A3D3E90023F6F7D0FC00220023E2
:1098E000F7F70EF950B1002C5ADA24F0004353EA8E
:1098F00008032F4B4FF0000518BF1C462146284691
:1099000025E02C4F374101EA070303431FD026A36C
:10991000D3E90023F6F7B2FC00220023F7F7F0F8B2
:109920000028EBD0002CBEBF4FF4801343FA06F69C
:10993000A41924EA07040025E0E7332E0BDDB6F571
:10994000806F04D110EE102A0B46F6F797FC41EC1D
:10995000100BBDE8F081A7F213474FF0FF3323FA55
:1099600007F73842F3D010A3D3E90023F6F786FCBB
:1099700000220023F7F7C4F80028BFD0002C02DA39
:10998000142E03D1013425EA0705B7E70123C6F1F8
:10999000340603FA06F63544A84588BFE418F2E712
:1099A00000252C46AAE700BF9C7500883CE4377E62
:1099B0000000F0BFFFFF0F0051EC100BF8B5C1F332
:1099C0000A55A5F2FF34132C0B460F4617DC002C6A
:1099D00009DA013401F0004303D143F07F5343F42B
:1099E0004013002128E0164A2241114200D180B1E3
:1099F0004FF4002323413B4423EA0203F1E7332CD5
:109A00000ADDB4F5806F04D110EE102A0B46F6F78C
:109A100035FC41EC100BF8BDA5F213424FF0FF35B9
:109A2000D5402842F5D0C4F133040122A2401218D7
:109A300028BF013322EA050108461946E9E700BFBD
:109A4000FFFF0F002DE9F04F2DED048B8DB057EC8B
:109A5000106B55EC114B00F06FF9AE4BB0EE408A35
:109A6000F0EE608A93F90090B9F1FF3F98465FD01D
:109A700022462B4620462946F7F74CF88346002815
:109A800056D132463B4630463946F7F743F8019007
:109A9000E8B10022002320462946F7F709F80028FC
:109AA00046D0012302939C4B03939C4BCDF828B0E6
:109AB0000022B9F1020FCDE90467CDE90645CDE9F1
:109AC000082333D002A800F008FF48BB5EE04FF047
:109AD000000A4FF0000B52465B4630463946F6F717
:109AE000E7FF4BEC19AB002855D052465B462046A9
:109AF0002946F6F7DDFF804618B301230293864B13
:109B00000393019B0A93CDE90467CDE90645CDE9AE
:109B100008ABB9F1000FD5D0804B0022CDE9082366
:109B20000A9B1BB1FFF772FA0A9B03609DED088B3D
:109B3000B0EE480AF0EE680A0DB0BDEC048BBDE84B
:109B4000F08F45EC104B00F0C0FE0028F0D05246DC
:109B50005B4620462946F6F7B5FF0028E8D00123EA
:109B600002936D4B03936B4BCDF8288093F9003033
:109B7000CDE90467CDE9064513B9CDE908ABA1E706
:109B800067490020CDE90801022B9BD1FFF73EFA7F
:109B900021230360C4E7B0EE480AF0EE680A00F043
:109BA00094FE0190002840F08A8047EC106B00F092
:109BB0008CFE002800F0838045EC104B00F085FE01
:109BC00000287CD053EC182B18EE100A1946F6F733
:109BD000A1FF98F90090504BB0B101220393019B73
:109BE00002920A93CDE90467CDE90645B9F1000F69
:109BF000C3D052465B4650465946F6F71BFEB9F1B4
:109C0000020FCDE90801C0E70322029203930A90F4
:109C1000CDE90467CDE90645B9F1000F2CD1414BE0
:109C20004FF06042CDE90823304652465B46394644
:109C3000F6F748FF002866D000223B4B2046294615
:109C4000F6F7CEFC04460D4645EC104B00F050FEF6
:109C5000204653EC102B2946F6F72AFF20B9334B48
:109C60004FF06042CDE9082398F90030022B4AD129
:109C7000FFF7CCF922238CE72D4B0022CDE90823F6
:109C8000304652465B463946F6F71CFF0028EBD0BB
:109C90000022254B20462946F6F7A2FC04460D4635
:109CA00045EC104B00F024FE204653EC102B2946C7
:109CB000F6F7FEFE0028D7D10022194BD2E700228A
:109CC000002351EC180BF6F7F3FE00283FF430AFF9
:109CD00047EC106B00F0F9FD00283FF429AF45EC8C
:109CE000104B00F0F2FD00283FF422AF0423029352
:109CF000094B039300230A93CDE90467CDE9064598
:109D00008DED089BB0E702A800F0E7FD00287FF486
:109D100007AFADE770000020F3AB00080000F03F94
:109D20000000F0FFFFFFEF470000E03FFFFFEFC73D
:109D30000000F07F000000002DE9F04F91B08DEDA4
:109D4000001B9DE8040257EC106B29F0004858EA0C
:109D5000020310EE10AA3D4600F0BD84784B27F0B8
:109D600000449C4209DC03D13EB9A0450DDC01E072
:109D7000984502DC98450ED16AB104F1404404F5DF
:109D8000801454EA0A0300F0A6846E4811B0BDE8BE
:109D9000F04F00F0A5BD002D53DA6B4B98454DDC1C
:109DA000A3F1547398454CDD4FEA2853A3F2FF33D7
:109DB000142B26DDC3F1340322FA03F101FA03F375
:109DC0009A423ED101F00101C1F1020B002A5BD1A0
:109DD0005B4B984524D104F1404303F5801353EACB
:109DE0000A0300F07884594B9C422DDDB9F1000F35
:109DF00080F275840020002141EC100B11B0BDE809
:109E0000F08F002A3ED1C3F1140348FA03F101FA9E
:109E100003F3984540F06B8401F00101C1F1020B9E
:109E20004B4B984518D1B9F1000F80F25C8448493A
:109E300032463B460020F6F7FDFCDDE74FF0020B13
:109E4000C4E74FF0000BC1E7B9F1000FD2DA9DE88B
:109E5000090003F10041CFE7B9F1804F06D1324646
:109E60003B4610461946F6F7BBFBC5E7394B99450B
:109E70000AD1002D08DB47EC106B11B0BDE8F04FA4
:109E800000F06CBC4FF0000B47EC106B00F016FDBF
:109E900051EC100BBAF1000F27D124B12C4B25F057
:109EA00040429A4221D1B9F1000F05DA02460B4631
:109EB00000202749F6F7BEFC002D9DDA04F140444E
:109EC00004F5801454EA0B0308D102460B461046F1
:109ED0001946F6F7D1F902460B46ACE7BBF1010F84
:109EE0008AD101F10043194686E7ED0F6B1E0D93F1
:109EF0005BEA030302D132463B46E8E7164B98453E
:109F000040F3FE8003F1047398450ADD0F4B9C4239
:109F10000DDCB9F1000FBFF66DAF07A3D3E9002345
:109F20009FE70E4B9C42F4DD094B9C4218DDB9F1D2
:109F3000000FF2DC5EE700BF9C7500883CE4377ED2
:109F40000000F07FC5AB0008FFFF3F43FFFFEF3F7E
:109F50000000F03F0000E03F0000E041FEFFEF3F67
:109F60000022634BF6F788F955A3D3E90023044692
:109F70000D46F6F735FB54A3D3E9002306460F46FA
:109F800020462946F6F72CFB0022CDE90201594B69
:109F900020462946F6F724FB02460B464CA1D1E9A0
:109FA0000001F6F769F922462B46F6F719FB02463F
:109FB0000B4600205049F6F75FF922462B468046B3
:109FC000894620462946F6F70BFB02460B464046DB
:109FD0004946F6F705FB40A3D3E90023F6F700FB5B
:109FE00002460B46DDE90201F6F746F902460B464A
:109FF00004460D4630463946F6F740F90020CDE9D3
:10A00000040132463B46F6F737F902460B46204636
:10A010002946F6F731F90D9A0BF1FF331343064643
:10A020000F4640F0EB819FED2E7BDDE900450024DB
:10A0300022462B46DDE900018DED027BF6F71CF987
:10A04000DDE90423F6F7CCFADDE9002380468946F2
:10A0500030463946F6F7C4FA02460B4640464946B2
:10A06000F6F70CF922462B4680468946DDE90401C5
:10A07000F6F7B6FA0B4604460D46024649464046F8
:10A08000CDE90045F6F7FAF81C4B994206460F4613
:10A090008B4640F3F78201F13F4303F5E0030343AE
:10A0A00000F0EA8110A3D3E90023DDE90201F6F70D
:10A0B00097FA0DA3D3E90023D5E600BFAFF30080E4
:10A0C000000000604715F73F44DF5DF80BAE543EDB
:10A0D000555555555555D53FFE822B654715F73FCC
:10A0E000000000000000F0BF9C7500883CE4377E53
:10A0F0000000F03F0000D03F0000E03FFFFF8F4036
:10A10000B4F5801F4FF0000205DAD34BF6F768FA7A
:10A110006FF034020C462315A3F2FF331344079368
:10A12000CE4BC4F3130444F07F559C4245F44015D4
:10A1300008DDCB4B9C4240F35E81079B01330793C4
:10A14000A5F580154FF0000A4FEACA030C930C9A4C
:10A15000C44B134493ED007B294653EC172B8DED34
:10A160000A7BCDE90801F6F787F8DDE90A23064600
:10A170000F46DDE90801F6F781F802460B4600209C
:10A18000B949F6F757FBCDE90E0102460B463046BA
:10A190003946F6F725FACDE90401DDE90434CDE9C5
:10A1A000023400230293DDE902896D1045F0005569
:10A1B00005F50025002205EB8A4340464946144632
:10A1C0001D46F6F70DFA02460B4630463946F6F7BD
:10A1D00053F8DDE90A2306460F4620462946F6F7DE
:10A1E0004BF802460B46DDE90801F6F745F8424612
:10A1F0004B46F6F7F5F902460B4630463946F6F778
:10A200003BF8DDE90E23F6F7EBF9DDE90423CDE9B0
:10A21000080110461946F6F7E3F97BA3D3E90023BA
:10A2200004460D46F6F7DCF979A3D3E90023F6F7E7
:10A2300025F822462B46F6F7D3F977A3D3E9002376
:10A24000F6F71CF822462B46F6F7CAF974A3D3E9B1
:10A250000023F6F713F822462B46F6F7C1F972A34E
:10A26000D3E90023F6F70AF822462B46F6F7B8F9A9
:10A270006FA3D3E90023F6F701F8224606460F46FE
:10A280002B4620462946F6F7ABF902460B463046E8
:10A290003946F6F7A5F9424604460D464B46DDE938
:10A2A0000401F5F7EBFFDDE90823F6F799F92246FB
:10A2B0002B46F5F7E3FF424606460F464B4640461F
:10A2C0004946F6F78DF90022684BCDE90A01F5F70A
:10A2D000D5FF32463B46F5F7D1FF02980D460446BE
:10A2E00002460B4640464946F6F77AF90022804678
:10A2F00089465E4B20462946F5F7BEFFDDE90A2375
:10A30000F5F7BAFF02460B4630463946F5F7B4FF7B
:10A31000DDE90423F6F764F9224606460F462B468C
:10A32000DDE90801F6F75CF902460B46304639468E
:10A33000F5F7A4FF06460F4602460B46404649463F
:10A34000F5F79CFF02983CA3D3E9002304460D4691
:10A35000F6F746F94246CDE908014B462046294624
:10A36000F5F78AFF02460B4630463946F5F784FF7B
:10A3700033A3D3E90023F6F733F933A3D3E900235A
:10A3800006460F4620462946F6F72AF902460B46AE
:10A3900030463946F5F772FF0C9A354B1344D3E932
:10A3A0000023F5F76BFF044607980D46F6F7B2F861
:10A3B0000C9A304B1344D3E9008906460F462246D7
:10A3C0002B46DDE90801F5F759FF42464B46F5F704
:10A3D00055FF32463B46F5F751FF029832463B4661
:10A3E000CDE90401F5F748FF42464B46F5F744FF37
:10A3F000DDE9082307E64FF0010AA5E69FED147B8F
:10A4000013E600BFAFF30080EF4E454A287ECA3FF7
:10A4100065DBC9934A86CD3F01411DA96074D13FD8
:10A420004D268F515555D53FFFAB6FDBB66DDB3FEA
:10A43000033333333333E33F000000E009C7EE3F1B
:10A44000FD033ADC09C7EE3FF5015B14E02F3EBE89
:10A45000000000000000F03F000040438E98030021
:10A4600079B60B00F8AB00080000F03F0000084090
:10A4700018AC000808AC0008B6A3D3E90023404696
:10A480004946F5F7FBFE2246CDE904012B4630464E
:10A490003946F5F7F1FE02460B46DDE90401F6F711
:10A4A0002FFB00287FF4FEADA54A2BF0004393421A
:10A4B00040F30C811B154FF4801AA3F2FE334AFAC5
:10A4C00003F35B44C3F30A529E4EA2F2FF321641DD
:10A4D000C3F3130A002023EA0601C2F114024AF46E
:10A4E000801A4AFA02FABBF1000F02460B462046D8
:10A4F0002946B8BFCAF1000AF5F7BEFECDE9000152
:10A5000042464B46DDE90001F5F7B8FE00207AA38C
:10A51000D3E9002304460D46F6F762F8DDE900238F
:10A5200006460F4620462946F5F7A6FE02460B468C
:10A5300040464946F5F7A0FE71A3D3E90023F6F79C
:10A540004FF871A3D3E90023804689462046294667
:10A55000F6F746F802460B4640464946F5F78EFEAA
:10A5600004460D4602460B4630463946F5F786FE50
:10A5700032463B4680468946F5F77EFE02460B464C
:10A5800020462946F5F778FE424606460F464B46DA
:10A5900040464946F6F724F85DA3D3E90023044674
:10A5A0000D46F6F71DF85CA3D3E90023F5F764FE2A
:10A5B00022462B46F6F714F859A3D3E90023F5F702
:10A5C0005DFE22462B46F6F70BF857A3D3E900238E
:10A5D000F5F752FE22462B46F6F702F854A3D3E9CC
:10A5E0000023F5F74BFE22462B46F5F7F9FF02460E
:10A5F0000B4640464946F5F73FFE04460D460246E7
:10A600000B4640464946F5F7EBFF0022CDE9000135
:10A610004FF0804320462946F5F72EFE02460B46B2
:10A62000DDE90001F6F706F9324604460D463B46E1
:10A6300040464946F5F7D4FF32463B46F5F71EFE45
:10A6400002460B4620462946F5F716FE42464B4683
:10A65000F5F712FE02460B4600203B49F5F70CFECB
:10A6600001EB0A54B4F5801F02460B4631DA50461E
:10A6700043EC102B00F0C4F951EC100BDDE9022380
:10A68000FFF7F1BB314B21F000469E427FF70CAF44
:10A690002F4B0B4403430BD027A3D3E90023DDE961
:10A6A0000201F5F79DFF24A3D3E90023FFF7DBBBED
:10A6B00022462B46F5F7E0FD02460B46404649464A
:10A6C000F6F70AFA00283FF4EFAEE5E74FF0000A8C
:10A6D00016E72146D2E700201B49FFF78DBBDDE9D5
:10A6E0000001FFF789BB30463946FFF785BB93462B
:10A6F000FFF796BBAFF3008000000000432EE63F5B
:10A70000EF39FAFE422EE63F396CA80C615C20BEA0
:10A71000D0A4BE726937663EF16BD2C541BDBB3E67
:10A720002CDE25AF6A56113F93BDBE166CC1663F45
:10A730003E5555555555C53F59F3F8C21F6EA501F5
:10A740000000E03FFFFF0F000000F03FFFCB904014
:10A7500000346F3FFE822B654715973C2DE9F04191
:10A7600055EC104B544EAE4310EE100A2B462A46C1
:10A77000214613D110EE102A2B4610EE100A29465E
:10A78000F5F72EFF02460B4620462946F5F776FDE3
:10A7900004460D4645EC104BBDE8F081002D10DC61
:10A7A00025F000463043F5D05DB110EE102A2B465F
:10A7B00020462946F5F760FD02460B46F6F73AF8C3
:10A7C000E6E71B150CD1002A6DD00020D6026ED50D
:10A7D000441E1B1BC0F1200421FA04F422438140D3
:10A7E000A3F2FF33C2F31302DD0742F4801242BF2B
:10A7F000520002EBD17249005810002502EBD173D0
:10A800001A44490016232C464FF40016A719974204
:10A81000DEBFD21BBC19AD195200013B02EBD17255
:10A820004FEA56064FEA4101F0D14FF0200E9C4608
:10A830004FF00046A24206EB0C0702DC12D18F4219
:10A8400010D8002F07EB060C34DABCF1000F31DB17
:10A8500004F10108121B8F4288BF02F1FF32C91BAD
:10A860003344444602EBD177BEF1010E3A444FEA3D
:10A8700041014FEA5606DDD10A4306D05C1C13BFE6
:10A8800001330135734623F001036A105B08E907C1
:10A8900002F17F5202F5001248BF43F0004302EB81
:10A8A00000551C4676E7CA0A153B49058BE752005E
:10A8B00001308BE7A046CDE70000F07F53EC102B72
:10A8C00023F0004343EC102B704710EE903A43F016
:10A8D000004000F58010C00F704700207047000056
:10A8E0009FED010B704700BF000000000000F87FE3
:10A8F000F7B551EC100BC1F30A54A4F2FF36132E36
:10A9000010EE107A0B4602464FEAD17558DC002E45
:10A910002BDA21F00042024323D0C1F31302024399
:10A9200051421143090B5B0C01F400215B0441EA25
:10A930000307314B03EBC5033946D3E9006710EE3B
:10A94000100A32463B46F5F799FCCDE900013B463B
:10A950003246DDE90001F5F78FFC21F0004343EAC0
:10A96000C57141EC100B03B0F0BD244C344101EA39
:10A9700004070743F5D0610803EA010002430BD046
:10A9800023EA01014FF48023132E43FA06F30CBF90
:10A990004FF0004200220B431946174B03EBC5054D
:10A9A000D5E9004510462B462246F5F767FCCDE970
:10A9B000000122462B46DDE90001F5F75DFCD0E7FA
:10A9C000332E08DDB6F5806FCBD110EE102A0B4682
:10A9D000F5F754FCC5E7A4F213464FF0FF34F440FA
:10A9E0002042BED061080F421FBF4FF0804227EACD
:10A9F000010132410A43CFE728AC0008FFFF0F00F6
:10AA000070B555EC104BC5F30A5206462B46B2B949
:10AA100025F0004323433CD00022334B294610EE5F
:10AA2000100AF5F7DDFD314A964204460D460B4605
:10AA300013DA29A3D3E90023F5F7D2FD0AE040F2A7
:10AA4000FF718A420CD110EE102A2B46204629466F
:10AA5000F5F714FC04460D461BE0C1F30A52363AE2
:10AA6000324440F2FE718A420BDD45EC114B9FED02
:10AA70001C0B00F03FF81AA3D3E9002351EC100B94
:10AA8000DAE7002A08DD23F0FF4323F4E00343EA7A
:10AA9000025545EC104B70BD12F1350F0DDA4CF23A
:10AAA00050339E4245EC114BE1DC9FED0B0B00F067
:10AAB00021F809A3D3E90023E0E723F0FF4336326E
:10AAC00023F4E00343EA0255204629460022084BBE
:10AAD000B2E700BFAFF3008059F3F8C21F6EA501C3
:10AAE0009C7500883CE4377E00005043B03CFFFF7B
:10AAF0000000903C53EC102B11EE900A23F0004123
:10AB000000F0004041EA000343EC102B70470000C6
:10AB1000F8B500BFF8BC08BC9E467047F8B500BF4A
:08AB2000F8BC08BC9E4670471A
:10AB280025356400313938373938323200000000B1
:10AB380030303030350000002447504747412C0062
:10AB480030303A30303A3030000000002020302ECB
:10AB58003030303030300000202020302E3030307F
:10AB68003030300020203000302E3000303030308F
:10AB7800303030302E30000020202020302E3000A1
:10AB880002030405060708090A0B0C0D0E0F101026
:10AB98000102030405060708090A0B0C0D0E0F1025
:10ABA8000000000000000000010203040607080975
:10ABB8000000000001020304232D302B2000686CE4
:10ABC8004C006566674546470030313233343536C8
:10ABD8003738394142434445460030313233343501
:10ABE8003637383961626364656600706F770000D4
:10ABF800000000000000F03F000000000000F83FE7
:10AC080000000000000000000000004003B8E23F20
:10AC1800000000000000000006D0CF43EBFD4C3ED2
:10AC2800000000000000304300000000000030C3B6
:08AC38009860FF7F010000009D
:04AC4000B501000852
:04AC44009101000872
:10AC4800100000000100000000127A00100000202F
:10AC580000000000000000000000000000000000EC
:10AC680000000000000000000000000000000000DC
:10AC780000000000000000000000000000000000CC
:10AC880000000000000000000000000000000000BC
:10AC980000000000000000000000000000000000AC
:10ACA800000000000000000000000000000000009C
:04ACB8000100000097
:0400000508008FB9A7
:00000001FF
